:030000000267AAEA
:1067AA00758E1190000078FF79FFE4F0A3D9FBD829
:0D67BA00F778FFE4F6D8FD75817C026802D7
:106ADE004401D240490FDB4401CE40C90FDB4401D3
:056AEE00CA3C8EFA35E0
:0646E4009001B2121F5EFE
:1046EA009001B6E0FCA3E0FDA3E0FEA3E0FFEF2407
:1046FA0069FFEE3474FEED34FFFDEC34FFFCEC127E
:10470A001AC87BDF7A927986783D1218A49001BA8A
:10471A00121F5E7B007A0079C078419001BAE0FCF2
:10472A00A3E0FDA3E0FEA3E0FF1219AD125F997B9F
:10473A00007A0079C078411218A4C004C005C006E6
:10474A00C0077F977E7E7DD57C409001BAE0F8A3B2
:10475A00E0F9A3E0FAA3E0FB1217B3D003D002D02A
:10476A0001D0001217AFC004C005C006C0077F926F
:10477A007E867DC07C419001B2E0F8A3E0F9A3E017
:10478A00FAA3E0FB1218A4A804A905AA06AB07D04D
:10479A0007D006D005D0041217B39001C2121F5ECB
:1047AA009001B6E0FCA3E0FDA3E0FEA3E0FFEF2446
:1047BA0069FFEE3474FEED34FFFDEC34FFFCEC12BD
:1047CA001AC89001B2E0F8A3E0F9A3E0FAA3E0FB6B
:1047DA001217B37B307AE67958783D1218A4A804E8
:1047EA00A905AA06AB077F817E0E7DBA7C43121704
:1047FA00AF9001CAE0F8A3E0F9A3E0FAA3E0FB1244
:10480A0018A49001BE121F5E9001CEE0FCA3E0FD49
:10481A00A3E0FEA3E0FF9001BEE0F8A3E0F9A3E065
:10482A00FAA3E0FB121A4A602940279001BEE0FC75
:10483A00A3E0FDA3E0FEA3E0FF9001CEE0F8A3E031
:10484A00F9A3E0FAA3E0FB1217AF9001BE121F5EB4
:10485A0080B69001CEE0FCA3E0FDA3E0FEA3E0FF5A
:10486A00121AB79001BEE0F8A3E0F9A3E0FAA3E0B8
:10487A00FB121A4A50279001BEE0FCA3E0FDA3E018
:10488A00FEA3E0FF9001CEE0F8A3E0F9A3E0FAA3CB
:10489A00E0FB1217B39001BE121F5E80B57F007E47
:1048AA00007D007C009001BEE0F8A3E0F9A3E0FAE5
:1048BA00A3E0FB121A4A604840469001D2E0FCA3EA
:1048CA00E0FDA3E0FEA3E0FF9001BEE0F8A3E0F95B
:1048DA00A3E0FAA3E0FB121A4A50259001BEE0FCBD
:1048EA00A3E0FDA3E0FEA3E0FF9001CEE0F8A3E081
:1048FA00F9A3E0FAA3E0FB1217AF9001BE121F5E04
:10490A007F007E007D007C009001BEE0F8A3E0F904
:10491A00A3E0FAA3E0FB121A4A504B9001D2E0FC42
:10492A00A3E0FDA3E0FEA3E0FF121AB79001BEE0E8
:10493A00F8A3E0F9A3E0FAA3E0FB121A4A602740C1
:10494A00259001BEE0FCA3E0FDA3E0FEA3E0FF90FA
:10495A0001CEE0F8A3E0F9A3E0FAA3E0FB1217B353
:10496A009001BE121F5E9001BEE0FCA3E0FDA3E031
:10497A00FEA3E0FF1256917B247A0B7998783912BC
:10498A0018A49001C2E0F8A3E0F9A3E0FAA3E0FBBF
:10499A001217B39001C6121F5E7B007A0079C078A5
:1049AA00419001C6E0FCA3E0FDA3E0FEA3E0FF12F4
:1049BA0019AD125F997B007A0079C078411218A468
:1049CA00A804A905AA06AB079001C6E0FCA3E0FD6E
:0949DA00A3E0FEA3E0FF1217AFF9
:0149E30022B1
:106A9C009001DD121F5E9001DDE0FCA3E0FDA3E0A0
:106AAC00FEA3E0FF125F99A804A905AA06AB079004
:106ABC0001DDE0FCA3E0FDA3E0FEA3E0FF1217AFB5
:106ACC009001CEE0F8A3E0F9A3E0FAA3E0FB1218E2
:026ADC00A422F2
:060C7D00900142121F5E0F
:100C8300900142E0FCA3E0FDA3E0FEA3E0FFEF241C
:100C930013FFEE342DFEED34FFFDEC34FFFCEC12BC
:100CA3001AC8900146E0F8A3E0F9A3E0FAA3E0FB39
:100CB3001217B390014A121F5E7F8D7EA67D147CAE
:100CC3003D90014AE0F8A3E0F9A3E0FAA3E0FB12A8
:100CD30018A47B807AF279BF783E1217B3126A9C0C
:100CE30090014E121F5E7F477E857D167C3D9001ED
:100CF3004AE0F8A3E0F9A3E0FAA3E0FB1218A47B0F
:100D0300937AA77984783E1217B3126A9C900152A2
:100D1300121F5E7F217EB47D0A7C3D90014AE0F87C
:100D2300A3E0F9A3E0FAA3E0FB1218A47BFF7ACDBA
:100D33007953783F1217B3126A9C900156121F5EC3
:100D43007F4D7E6C7D337C3B90014AE0F8A3E0F954
:100D5300A3E0FAA3E0FB1218A47B817A3D797E78A5
:100D63003F1217B3126A9C90015A121F5E7F007ED6
:100D7300007D007C40900156E0F8A3E0F9A3E0FA7F
:100D8300A3E0FB1218A4A804A905AA06AB079001C7
:100D93004EE0FCA3E0FDA3E0FEA3E0FF1217AF12B9
:100DA300567B7BF37A767914783F1218A4C004C07B
:100DB30005C006C00790014EE0FCA3E0FDA3E0FEE2
:100DC300A3E0FF12567B7BE87AC179517840121871
:100DD300A4A804A905AA06AB077FB17E737D717C25
:100DE300421217AFD003D002D001D0001217AFC008
:100DF30004C005C006C0077F007E007D007C4090D4
:100E03000156E0F8A3E0F9A3E0FAA3E0FB1218A46B
:100E130012567B7B0C7A5979ED783E1218A4A804FC
:100E2300A905AA06AB07D007D006D005D004121730
:100E3300AF90015E121F5E7F007E007D007C4090BC
:100E43000156E0F8A3E0F9A3E0FAA3E0FB1218A42B
:100E5300C004C005C006C0077F007E007D007C4043
:100E630090014EE0F8A3E0F9A3E0FAA3E0FB121827
:100E7300A4D003D002D001D0001217AF12567B7B4F
:100E8300767A4F791E783D1218A4C004C005C006B7
:100E9300C0077F007E007D007C4090014EE0F8A3F8
:100EA300E0F9A3E0FAA3E0FB1218A412567B7B9CA3
:100EB3007A5A79B6783D1218A4A804A905AA06ABF4
:100EC3000790015EE0FCA3E0FDA3E0FEA3E0FF12B8
:100ED30017AFA804A905AA06AB07D007D006D0050B
:100EE300D0041217B3C004C005C006C0077F007E3C
:100EF300007D007C40900156E0F8A3E0F9A3E0FAFE
:100F0300A3E0FB1218A490015AE0F8A3E0F9A3E0D0
:100F1300FAA3E0FB1217AF12567B7B687A9679042B
:100F2300783D1218A4A804A905AA06AB07D007D0D8
:100F330006D005D0041217AF90015E121F5E7F002A
:100F43007E007D007C40900156E0F8A3E0F9A3E029
:100F5300FAA3E0FB1218A4A804A905AA06AB0790FC
:100F6300014EE0FCA3E0FDA3E0FEA3E0FF1217AFF8
:100F730090015AE0F8A3E0F9A3E0FAA3E0FB12170B
:100F8300B312567B7BD87A2A79C1783C1218A4C055
:100F930004C005C006C0077F007E007D007C409032
:100FA3000156E0F8A3E0F9A3E0FAA3E0FB1218A4CA
:100FB300A804A905AA06AB0790014EE0FCA3E0FD37
:100FC300A3E0FEA3E0FF1217AF12567B7B727A33C6
:100FD30079DC783C1218A4A804A905AA06AB0790EB
:100FE300015EE0FCA3E0FDA3E0FEA3E0FF1217AF68
:100FF300D003D002D001D0001217AFC004C005C087
:1010030006C00790015AE0F8A3E0F9A3E0FAA3E0D1
:10101300FB90014EE0FCA3E0FDA3E0FEA3E0FF1282
:1010230017AF12567B7B307A4C79A6783C1218A402
:10103300A804A905AA06AB07D007D006D005D0049B
:101043001217AF90015E121F5E900156E0FCA3E001
:10105300FDA3E0FEA3E0FF12567B7B0B7AD2798CD3
:10106300783C1218A490015EE0F8A3E0F9A3E0FA3B
:10107300A3E0FB1217B3C004C005C006C00790016C
:101083005AE0FCA3E0FDA3E0FEA3E0FF90014EE0E5
:10109300F8A3E0F9A3E0FAA3E0FB1217B312567B1F
:1010A3007B697AE37988783C1218A4A804A905AA75
:1010B30006AB07D007D006D005D0041217B39001B2
:1010C3005E121F5E7F007E007D007C40900152E037
:1010D300F8A3E0F9A3E0FAA3E0FB1218A4A804A97B
:1010E30005AA06AB0790014EE0FCA3E0FDA3E0FEDA
:1010F300A3E0FF1217AF12567B7BF97A4E794C7837
:101103003C1218A4C004C005C006C00790015AE0F1
:10111300FCA3E0FDA3E0FEA3E0FF12567B7BCD7AA8
:10112300AF79E6783B1218A4A804A905AA06AB0771
:10113300D007D006D005D0041217B3C004C005C031
:1011430006C0077F007E007D007C40900156E0F8DA
:10115300A3E0F9A3E0FAA3E0FB1218A490015AE07C
:10116300F8A3E0F9A3E0FAA3E0FB1217B312567B4E
:101173007BBC7A5779AD783B1218A4A804A905AAB9
:1011830006AB07D007D006D005D0041217B3C004AE
:10119300C005C006C0077F007E007D807C409001B3
:1011A30056E0F8A3E0F9A3E0FAA3E0FB1218A4A821
:1011B30004A905AA06AB0790014EE0FCA3E0FDA33A
:1011C300E0FEA3E0FF1217AF12567B7B4E7AB47991
:1011D300AB783B1218A4A804A905AA06AB07D0074D
:1011E300D006D005D0041217AF900162121F5E7FA4
:1011F300007E007D007C40900156E0F8A3E0F9A357
:10120300E0FAA3E0FB1218A4A804A905AA06AB07F9
:1012130090014EE0FCA3E0FDA3E0FEA3E0FF121764
:10122300AF90015AE0F8A3E0F9A3E0FAA3E0FB12C0
:1012330017AF12567B7BA97A6A7982783B1218A47E
:10124300900162E0F8A3E0F9A3E0FAA3E0FB121730
:10125300B3C004C005C006C0077F007E007D407C8C
:101263004090014EE0F8A3E0F9A3E0FAA3E0FB12FB
:1012730018A412567B7B9C7ADC796F783B1218A4F6
:10128300A804A905AA06AB07D007D006D005D00449
:101293001217AFC004C005C006C0077F007E007DE3
:1012A300807C40900156E0F8A3E0F9A3E0FAA3E0C4
:1012B300FB1218A4C004C005C006C0077F007E004F
:1012C3007D007C4090014EE0F8A3E0F9A3E0FAA38F
:1012D300E0FB1218A4D003D002D001D0001217AF44
:1012E30012567B7BCA7A547941783B1218A4A8041E
:1012F300A905AA06AB07D007D006D005D00412175C
:10130300AF900162121F5E7F007E007D007C4090E3
:101313000156E0F8A3E0F9A3E0FAA3E0FB1218A456
:10132300C004C005C006C0077F007E007D407C402E
:1013330090014EE0F8A3E0F9A3E0FAA3E0FB121852
:10134300A4D003D002D001D0001217AF12567B7B7A
:10135300457A2F7923783B1218A4C004C005C00630
:10136300C00790015AE0FCA3E0FDA3E0FEA3E0FF69
:10137300900156E0F8A3E0F9A3E0FAA3E0FB12170B
:10138300B312567B7B147A5C792C783B1218A4A891
:1013930004A905AA06AB07900162E0FCA3E0FDA344
:1013A300E0FEA3E0FF1217AFA804A905AA06AB0746
:1013B300D007D006D005D0041217B3C004C005C0AF
:1013C30006C0077F007E007D007C40900156E0F858
:1013D300A3E0F9A3E0FAA3E0FB1218A490014EE006
:1013E300F8A3E0F9A3E0FAA3E0FB1217B390015AC4
:1013F300E0F8A3E0F9A3E0FAA3E0FB1217AF12565B
:101403007B7BA67AD57910783B1218A4A804A9058A
:10141300AA06AB07D007D006D005D0041217AFC079
:1014230004C005C006C0077F007E007D007C40909D
:101433000156E0F8A3E0F9A3E0FAA3E0FB1218A435
:10144300C004C005C006C0077F007E007D007C404D
:10145300900152E0F8A3E0F9A3E0FAA3E0FB12182D
:10146300A4D003D002D001D0001217AF12567B7B59
:10147300B37A7B79F2783A1218A4A804A905AA06CC
:10148300AB07D007D006D005D0041217B390016282
:10149300121F5E7F007E007D007C40900152E0F8C9
:1014A300A3E0F9A3E0FAA3E0FB1218A490014EE035
:1014B300F8A3E0F9A3E0FAA3E0FB1217B3C004C05A
:1014C30005C006C0077F007E007D007C409001566A
:1014D300E0F8A3E0F9A3E0FAA3E0FB1218A4A80440
:1014E300A905AA06AB07D007D006D005D00412176A
:1014F300AF12567B7B047AAD79C0783A1218A4C038
:1015030004C005C006C0077F007E007D007C4090BC
:10151300015AE0F8A3E0F9A3E0FAA3E0FB1218A450
:10152300C004C005C006C0077F007E007D007C406C
:10153300900156E0F8A3E0F9A3E0FAA3E0FB121848
:10154300A4D003D002D001D0001217AF12567B7B78
:10155300A37A0679D378BA1218A4A804A905AA060F
:10156300AB07D007D006D005D0041217B3C004C010
:1015730005C006C0077F007E007D807C4090015639
:10158300E0F8A3E0F9A3E0FAA3E0FB1218A41256D3
:101593007B7B4B7A1F79BA783A1218A4A804A90561
:1015A300AA06AB07D007D006D005D0041217AFC0E8
:1015B30004C005C006C0077F007E007D007C40900C
:1015C3000156E0F8A3E0F9A3E0FAA3E0FB1218A4A4
:1015D300C004C005C006C0077F007E007D007C40BC
:1015E30090014EE0F8A3E0F9A3E0FAA3E0FB1218A0
:1015F300A4D003D002D001D0001217AF90015AE05B
:10160300F8A3E0F9A3E0FAA3E0FB1217B312567BA9
:101613007BA97A3079B6783A1218A4A804A905AA46
:1016230006AB07D007D006D005D0041217B390013C
:1016330066121F5E7F007E007D807C40900156E035
:10164300F8A3E0F9A3E0FAA3E0FB1218A4A804A905
:1016530005AA06AB0790014EE0FCA3E0FDA3E0FE64
:10166300A3E0FF1217AF90015AE0F8A3E0F9A3E05B
:10167300FAA3E0FB1217B312567B7B3B7AAA799A43
:10168300783A1218A4A804A905AA06AB0790016624
:10169300E0FCA3E0FDA3E0FEA3E0FF1217AFC0044C
:1016A300C005C006C0077F007E007D007C4090011E
:1016B30056E0F8A3E0F9A3E0FAA3E0FB1218A4C0F4
:1016C30004C005C006C0077F007E007D007C4090FB
:1016D300014EE0F8A3E0F9A3E0FAA3E0FB1218A49B
:1016E300A804A905AA06AB07D007D006D005D004E5
:1016F3001217B312567B7B247A0B7998783A121817
:10170300A4A804A905AA06AB07D007D006D005D024
:10171300041217AFC004C005C006C0077F007E00D7
:101723007D007C4090014EE0F8A3E0F9A3E0FAA32A
:10173300E0FB1218A490015AE0F8A3E0F9A3E0FA41
:10174300A3E0FB1217AF12567B7BE07A2D799078DA
:101753003A1218A4A804A905AA06AB07D007D00615
:10176300D005D0041217AF900166121F5E9001627C
:10177300E0FCA3E0FDA3E0FEA3E0FF90015EE0F840
:10178300A3E0F9A3E0FAA3E0FB1217B3900166E02C
:10179300F8A3E0F9A3E0FAA3E0FB1217B37B487ABE
:0817A3005179C778451218A422
:0117AB00221B
:0B29D500900108EBF0A3EAF0A3E9F08A
:1029E00090010EE0FCA3E0FDA3E0FEA3E0FFEC12EB
:1029F0001AC87B007A81798878C61217B3900112C1
:102A0000E0F8A3E0F9A3E0FAA3E0FB1217B390010A
:102A100016121F5E7F0A7EEB7D157C3D900116E04D
:102A2000F8A3E0F9A3E0FAA3E0FB1218A47B7F7AF5
:102A30004F7940783F1217B3126A9C90011A121F07
:102A40005E7F8C7EA67D147C3D900116E0F8A3E0AD
:102A5000F9A3E0FAA3E0FB1218A47B367A9079522E
:102A6000783F1217B3126A9C90011E121F5E7F4DB1
:102A70007E6C7D337C3B900116E0F8A3E0F9A3E087
:102A8000FAA3E0FB1218A47B857AEA797E783F12DC
:102A900017B3126A9C900122121F5E7F217EB47DC3
:102AA0000A7C3D900116E0F8A3E0F9A3E0FAA3E068
:102AB000FB1218A47BD37A697979783F1217B31285
:102AC0006A9C900126121F5E7F477E857D167C3DA5
:102AD000900116E0F8A3E0F9A3E0FAA3E0FB1218D6
:102AE000A47B9F7A027900783D1217B3126A9C90FA
:102AF000012A121F5E7F007E007D007C409001262F
:102B0000E0F8A3E0F9A3E0FAA3E0FB1218A4125640
:102B1000917BB07A727928783F1218A4C004C0055E
:102B2000C006C00790011EE0FCA3E0FDA3E0FEA3E9
:102B3000E0FF1256917B7D7A3F79C978401218A444
:102B4000A804A905AA06AB07D007D006D005D00473
:102B50001217B3C004C005C006C0077F007E007D09
:102B6000007C40900126E0F8A3E0F9A3E0FAA3E09E
:102B7000FB1218A4A804A905AA06AB0790011EE041
:102B8000FCA3E0FDA3E0FEA3E0FF1217AF125691F5
:102B90007B6F7A1279A3783F1218A4A804A905AA1A
:102BA00006AB07D007D006D005D0041217AFC0047B
:102BB000C005C006C007900122E0FCA3E0FDA3E031
:102BC000FEA3E0FF1256917BC97A76793E783E12D9
:102BD00018A4A804A905AA06AB07D007D006D005FB
:102BE000D0041217AF9001CAE0F8A3E0F9A3E0FA0D
:102BF000A3E0FB1218A490011AE0F8A3E0F9A3E007
:102C0000FAA3E0FB1217B390012E121F5E90012E63
:102C1000E0FCA3E0FDA3E0FEA3E0FFC004C005C00C
:102C200006C0077F007E007D007C4090012AE0F80E
:102C3000A3E0F9A3E0FAA3E0FB1218A41256917BDB
:102C4000D57A7879E9783D1218A4C004C005C00689
:102C5000C0077F007E007D007C4090011EE0F8A34D
:102C6000E0F9A3E0FAA3E0FB1218A41256917BD17D
:102C70007A22795B783E1218A4D003D002D001D01A
:102C8000001217AFC004C005C006C0077F007E0059
:102C90007D007C40900126E0F8A3E0F9A3E0FAA3D0
:102CA000E0FB1218A4C004C005C006C0077F007E68
:102CB000007D007C4090011EE0F8A3E0F9A3E0FA5B
:102CC000A3E0FB1218A4D003D002D001D000121749
:102CD000AF1256917BFC7AA97971783D1218A4A89D
:102CE00004A905AA06AB07D007D006D005D0041268
:102CF00017AFC004C005C006C0077F007E007D007E
:102D00007C40900126E0F8A3E0F9A3E0FAA3E0FB01
:102D10001218A4C004C005C006C007900122E0FC40
:102D2000A3E0FDA3E0FEA3E0FF90011EE0F8A3E016
:102D3000F9A3E0FAA3E0FB1217B3D003D002D0014D
:102D4000D0001217AF1256917BD57A787969783D09
:102D50001218A4A804A905AA06AB07D007D006D06C
:102D600005D0041217AF9001CAE0F8A3E0F9A3E080
:102D7000FAA3E0FB1218A4A804A905AA06AB07D081
:102D800007D006D005D0041217B390012E121F5E93
:102D90007F007E007D007C40900126E0F8A3E0F9F2
:102DA000A3E0FAA3E0FB1218A41256917BE37AC7C2
:102DB0007928783F1218A4C004C005C006C0079047
:102DC000011EE0FCA3E0FDA3E0FEA3E0FF1256918C
:102DD0007B9E7A5E79C778401218A4A804A905AA38
:102DE00006AB07D007D006D005D0041217B3C00435
:102DF000C005C006C0077F007E007D007C409001BA
:102E000026E0F8A3E0F9A3E0FAA3E0FB1218A4A8D7
:102E100004A905AA06AB0790011EE0FCA3E0FDA3F0
:102E2000E0FEA3E0FF1217AF1256917BE57AD0794E
:102E3000A2783F1218A4A804A905AA06AB07D007D8
:102E4000D006D005D0041217AF9001CAE0F8A3E075
:102E5000F9A3E0FAA3E0FB1218A490012AE0F8A37A
:102E6000E0F9A3E0FAA3E0FB1217B3900132121FBE
:102E70005E7F007E007D007C40900126E0F8A3E0AC
:102E8000F9A3E0FAA3E0FB1218A4A804A905AA0676
:102E9000AB0790012AE0FCA3E0FDA3E0FEA3E0FF66
:102EA0001217AF1256917B067A817915783E121867
:102EB000A4C004C005C006C007900132E0FCA3E036
:102EC000FDA3E0FEA3E0FF1256917BA67A9B79A4B6
:102ED00078401218A4D003D002D001D0001217AF4E
:102EE0009001CAE0F8A3E0F9A3E0FAA3E0FB12180E
:102EF000A4900136121F5E90012EE0FCA3E0FDA31A
:102F0000E0FEA3E0FF125691C004C005C006C00752
:102F1000900136E0FCA3E0FDA3E0FEA3E0FF125623
:102F20007BA804A905AA06AB07D007D006D005D018
:102F3000041218A47B327AAF79CB783E1218A4C061
:102F400004C005C006C007900136E0FCA3E0FDA365
:102F5000E0FEA3E0FF1256917BDB7ADE796A783FD0
:102F60001218A4A804A905AA06AB07D007D006D05A
:102F700005D0041217B390010BE0FBA3E0FAA3E025
:102F8000F9121EEC90010BE0FBA3E0FAA3E0F912AA
:102F90001ECC90010BE0FBA3E0FAA3E0F9121F3E68
:102FA0001218A4A804A905AA06AB077F007E007D1D
:102FB000807C3F1217AF1265BA9000D0121F5E904E
:102FC000010BE0FBA3E0FAA3E0F9121ECC12684764
:102FD00090010BE0FBA3E0FAA3E0F9121EEC9001D4
:102FE0002EE0FCA3E0FDA3E0FEA3E0FF12567BC0B1
:102FF00004C005C006C007900136E0FCA3E0FDA3B5
:10300000E0FEA3E0FF12567BA804A905AA06AB07C1
:10301000D007D006D005D0041218A4C004C005C043
:1030200006C00790010BE0FBA3E0FAA3E0F9121E33
:10303000CC12567BA804A905AA06AB07D007D00678
:10304000D005D0041219AD90013A121F5E90012EE6
:10305000E0FCA3E0FDA3E0FEA3E0FF125691C00454
:10306000C005C006C007900136E0FCA3E0FDA3E068
:10307000FEA3E0FF12567BA804A905AA06AB07D061
:1030800007D006D005D0041218A47BDB7ADE796A5B
:10309000783F1218A4C004C005C006C007900136CE
:1030A000E0FCA3E0FDA3E0FEA3E0FF1256917B321B
:1030B0007AAF79CB783E1218A4A804A905AA06AB6A
:1030C00007D007D006D005D0041217AFC004C00542
:1030D000C006C00790010BE0FBA3E0FAA3E0F912E1
:1030E0001ECC12567BA804A905AA06AB07D007D0B0
:1030F00006D005D0041219AD90013E121F5E90015A
:103100003EE0FCA3E0FDA3E0FEA3E0FFC004C00599
:10311000C006C00790013AE0FCA3E0FDA3E0FEA3D7
:10312000E0FF9000D0121F5ED007D006D005D0047B
:10313000126847900108E0FBA3E0FAA3E0F9121E31
:10314000EC900108E0FBA3E0FAA3E0F9121ECC7BAF
:10315000007A0079007800121A4A6030402E9001FF
:1031600008E0FBA3E0FAA3E0F9C003C002C001122B
:103170001ECC9001CEE0F8A3E0F9A3E0FAA3E0FBB7
:103180001217B3D001D002D003121EEC900108E058
:10319000FBA3E0FAA3E0F9121ECC9001CEE0F8A365
:1031A000E0F9A3E0FAA3E0FB121A4A502E900108BE
:1031B000E0FBA3E0FAA3E0F9C003C002C001121EC5
:1031C000CC9001CEE0F8A3E0F9A3E0FAA3E0FB1273
:0B31D00017AFD001D002D003121EEC9C
:0131DB0022D1
:0B3FC100900190EBF0A3EAF0A3E9F000
:103FCC00900196E0FCA3E0FDA3E0FEA3E0FFEC1261
:103FDC001AC87B007A81798878C61217B390019A37
:103FEC00E0F8A3E0F9A3E0FAA3E0FB1217B37B001F
:103FFC007AAD790E78471219AD90019E121F5E7F33
:10400C00A67EFE7DC77C4290019EE0F8A3E0F9A35A
:10401C00E0FAA3E0FB1218A47B917AEA797E783F50
:10402C001217B3126A9C9001A2121F5E7F117E239D
:10403C007D5F7C3790019EE0F8A3E0F9A3E0FAA342
:10404C00E0FB1218A4A804A905AA06AB077F507EB2
:10405C00AC7DAE7C3B1217AF126A9CC004C005C08D
:10406C0006C0079001A2E0FCA3E0FDA3E0FEA3E0E4
:10407C00FF125691A804A905AA06AB07D007D006D3
:10408C00D005D0041218A4C004C005C006C0077F18
:10409C00187E017DC87C4290019EE0F8A3E0F9A354
:1040AC00E0FAA3E0FB1218A47B327AE47946783F5D
:1040BC001217B3126A9CA804A905AA06AB07D0076D
:1040CC00D006D005D0041217B3C004C005C006C07A
:1040DC00077F007E007D007C409001A2E0F8A3E009
:1040EC00F9A3E0FAA3E0FB1218A41256917B0C7A08
:1040FC0034796978381218A4A804A905AA06AB0764
:10410C00D007D006D005D0041217B39001A6121F09
:10411C005E7F147E6A7D177C3890019EE0F8A3E0E8
:10412C00F9A3E0FAA3E0FB1218A4A804A905AA06B7
:10413C00AB077F6D7E6A7D857C3D1217AF126A9C42
:10414C009001AA121F5E9001A6E0FCA3E0FDA3E083
:10415C00FEA3E0FF1256CDC004C005C006C00790F8
:10416C0001AAE0FCA3E0FDA3E0FEA3E0FF12567B56
:10417C00A804A905AA06AB07D007D006D005D00421
:10418C001218A4125B82900190E0FBA3E0FAA3E06A
:10419C00F9121EEC9001CEE0F8A3E0F9A3E0FAA32B
:1041AC00E0FB9001A6E0FCA3E0FDA3E0FEA3E0FF92
:1041BC001219AD125F999001CEE0F8A3E0F9A3E0DB
:1041CC00FAA3E0FB1218A4A804A905AA06AB079051
:1041DC0001A6E0FCA3E0FDA3E0FEA3E0FF1217AFF5
:1041EC009001AE121F5E7F007E007DC07C3F90016F
:1041FC00D2E0F8A3E0F9A3E0FAA3E0FB1218A49034
:10420C0001AEE0F8A3E0F9A3E0FAA3E0FB121A4A2E
:10421C00505A7F007E007D007C3F9001D2E0F8A3D5
:10422C00E0F9A3E0FAA3E0FB1218A49001AEE0F8C9
:10423C00A3E0F9A3E0FAA3E0FB121A4A402E900186
:10424C0090E0FBA3E0FAA3E0F9C003C002C00112A6
:10425C001ECC9001D2E0F8A3E0F9A3E0FAA3E0FBB6
:10426C001217B3D001D002D003121EEC900190E0D3
:10427C00FBA3E0FAA3E0F9C003C002C001121ECCFC
:10428C00C004C005C006C007900190E0FBA3E0FA93
:10429C00A3E0F9121ECC9001CEE0F8A3E0F9A3E064
:1042AC00FAA3E0FB1219AD125F999001CEE0F8A3CE
:1042BC00E0F9A3E0FAA3E0FB1218A4A804A905AA4C
:1042CC0006AB07D007D006D005D0041217AFD0012B
:1042DC00D002D003121EEC9001A6E0FCA3E0FDA3DB
:1042EC00E0FEA3E0FF125691C004C005C006C00753
:1042FC009001AAE0FCA3E0FDA3E0FEA3E0FF1256B0
:10430C0091A804A905AA06AB07D007D006D005D002
:10431C00041218A4900193E0FBA3E0FAA3E0F912B5
:10432C001EEC900193E0FBA3E0FAA3E0F9121ECC83
:10433C00900193E0FBA3E0FAA3E0F9121F3E1218E0
:10434C00A4A804A905AA06AB077F007E007D807C8B
:10435C003F1217AF1265BA9000D0121F5E900193F6
:10436C00E0FBA3E0FAA3E0F9121ECC12684790011F
:0C437C0093E0FBA3E0FAA3E0F9121EECB2
:014388002212
:0B31DC0090016AEBF0A3EAF0A3E9F019
:1031E7007F927E0A7D867C3E900170E0F8A3E0F92D
:1031F700A3E0FAA3E0FB1218A4900174E0F8A3E09F
:10320700F9A3E0FAA3E0FB1217AF90017C121F5E4F
:103217007F007E007D007C0090017CE0F8A3E0F950
:10322700A3E0FAA3E0FB121A4A502790017CE0FCC6
:10323700A3E0FDA3E0FEA3E0FF9001CEE0F8A3E04A
:10324700F9A3E0FAA3E0FB1217B390017C121F5E0B
:1032570080489001CEE0FCA3E0FDA3E0FEA3E0FFE1
:1032670090017CE0F8A3E0F9A3E0FAA3E0FB121ACF
:103277004A6027402590017CE0FCA3E0FDA3E0FE27
:10328700A3E0FF9001CEE0F8A3E0F9A3E0FAA3E002
:10329700FB1217AF90017C121F5E90017CE0F8A330
:1032A700E0F9A3E0FAA3E0FB90001EE0FCA3E0FD39
:1032B700A3E0FEA3E0FF1217AF900016121F5E9067
:1032C7000016E0FCA3E0FDA3E0FEA3E0FF12567B9F
:1032D700C004C005C006C00790001AE0FCA3E0FDCB
:1032E700A3E0FEA3E0FF12567BA804A905AA06AB3C
:1032F70007D007D006D005D0041218A4C004C00513
:10330700C006C007900178E0FCA3E0FDA3E0FEA3A0
:10331700E0FF12567BA804A905AA06AB07D007D081
:1033270006D005D0041218A4C004C005C006C00703
:1033370090001AE0FCA3E0FDA3E0FEA3E0FF125615
:1033470091C004C005C006C007900178E0FCA3E067
:10335700FDA3E0FEA3E0FF125691A804A905AA0663
:10336700AB07D007D006D005D0041218A4A804A92B
:1033770005AA06AB07D007D006D005D0041217B3AD
:10338700900180121F5E900180E0FCA3E0FDA3E0A6
:10339700FEA3E0FF900180E0F8A3E0F9A3E0FAA321
:1033A700E0FB1218A4A804A905AA06AB077F007EB4
:1033B700007D807C3F1217AF1265BA900184121FFF
:1033C7005E900180E0FCA3E0FDA3E0FEA3E0FFC068
:1033D70004C005C006C007900184E0FCA3E0FDA37C
:1033E700E0FEA3E0FF9000D0121F5ED007D006D00A
:1033F70005D00412684790016DE0FBA3E0FAA3E053
:10340700F9121EEC90016DE0FBA3E0FAA3E0F912BC
:103417001ECC12567BC004C005C006C00790016DC4
:10342700E0FBA3E0FAA3E0F9121ECC125691D003F9
:10343700D002D001D0001219ADC004C005C006C02B
:103447000790001AE0FCA3E0FDA3E0FEA3E0FF1253
:10345700567BC004C005C006C00790001AE0FCA355
:10346700E0FDA3E0FEA3E0FF125691D003D002D007
:1034770001D0001219ADA804A905AA06AB07D00709
:10348700D006D005D0041218A4C004C005C006C0D9
:103497000790016DE0FBA3E0FAA3E0F9121ECC123E
:1034A700567BC004C005C006C00790001AE0FCA305
:1034B700E0FDA3E0FEA3E0FF12567BA804A905AA3E
:1034C70006AB07D007D006D005D0041218A4C00455
:1034D700C005C006C007900178E0FCA3E0FDA3E0AB
:1034E700FEA3E0FF125691D003D002D001D0001204
:1034F70019ADD003D002D001D0001217AF90018CC4
:10350700121F5E900178E0FCA3E0FDA3E0FEA3E0BC
:10351700FF12567BC004C005C006C00790001AE022
:10352700FCA3E0FDA3E0FEA3E0FF12567BA804A9DD
:1035370005AA06AB07D007D006D005D0041218A4F9
:10354700C004C005C006C007900016E0FCA3E0FD5C
:10355700A3E0FEA3E0FF12567BA804A905AA06ABC9
:1035670007D007D006D005D0041218A4C004C005A0
:10357700C006C007900178E0FCA3E0FDA3E0FEA32E
:10358700E0FF125691C004C005C006C00790001A9C
:10359700E0FCA3E0FDA3E0FEA3E0FF125691A80420
:1035A700A905AA06AB07D007D006D005D004121884
:1035B700A4A804A905AA06AB07D007D006D005D052
:1035C700041217B3900188121F5E900178E0FCA3E4
:1035D700E0FDA3E0FEA3E0FF12567BC004C005C0D8
:1035E70006C007900016E0FCA3E0FDA3E0FEA3E001
:1035F700FF125691A804A905AA06AB07D007D00663
:10360700D005D0041218A4C004C005C006C0079096
:103617000188E0FCA3E0FDA3E0FEA3E0FF900188A2
:10362700E0F8A3E0F9A3E0FAA3E0FB1218A4A804CA
:10363700A905AA06AB077F007E007D807C3F121795
:10364700AF1265BAA804A905AA06AB07D007D0062A
:10365700D005D0041219AD900188121F5E90018821
:10366700E0FCA3E0FDA3E0FEA3E0FFC004C005C0AB
:1036770006C00790018CE0FCA3E0FDA3E0FEA3E0F9
:10368700FF9000D0121F5ED007D006D005D00412DD
:10369700684790016AE0FBA3E0FAA3E0F9121EEC89
:1036A70090016AE0FBA3E0FAA3E0F9121ECC7B00CD
:1036B7007A0079007800121A4A6030402E90016A29
:1036C700E0FBA3E0FAA3E0F9C003C002C001121EA9
:1036D700CC9001CEE0F8A3E0F9A3E0FAA3E0FB1257
:0B36E70017B3D001D002D003121EEC7C
:0136F20022B5
:10650A00323B171C0205006400640001000007A367
:10651A00008703840064070803840682056900076C
:10652A0000020009003B003B0017001C000C00633E
:10653A0000C700C70002000A0E0F03840E0F03846F
:10654A000E0F07080E0F070800080005000E0000CE
:10655A00000000000001000100000001000100002D
:10656A000000000000000000000000000000000021
:10657A00000000000000000000000003000000030B
:10658A0000020003000200030003000200030002ED
:10659A0000030000000300010003000200030002E0
:0C65AA00000300030002000300020003D5
:066AF300C112C114C11321
:106975009000107432F0900011743BF09000127486
:1069850017F0900013741CF09000147402F090003E
:10699500157405F0124CC1756E00756F00D3E56F67
:1069A500940EE56E64809480503CE56F25E0FFE52C
:1069B5006E33FE74102FF58274653EF583E493FC07
:1069C500740193FDE56F25E0FFE56E33FE74222F1C
:1069D500F58274003EF583ECF0A3EDF0056FE56FED
:0A69E5007002056E80B7124DC52246
:103B760090003FE0F569D3E56964809482400BC309
:103B8600E569648094865002C212E5A064FFFFEFE7
:103B96005407F56BE56B6006C29CC2988002D29C06
:103BA600E56B5406FFEF6027056DE56DD3940A407B
:103BB6000F756A0AC3E569648094865003756D0AB9
:103BC600E56DD39414400E756A64756D14800675A0
:103BD6006D00756A01AF69EF3395E0FEEF25E0FFF2
:103BE600EE33FE74582FF58274653EF583E493F543
:103BF60067740193F568AF69EF3395E0FEEF25E052
:103C0600FFEE33FE742E2FF58274653EF583E49342
:103C1600F565740193F566E5696403706B900015AC
:103C2600E0FFEF75F004121D86AFF0EF602E9000F6
:103C360014E0FFEF3395E0FEEF25E0FFEE33FE7470
:103C4600822FF58274653EF583E493FE740193FF3B
:103C5600EF2566F566EE3565F565802C900014E077
:103C6600FFEF3395E0FEEF25E0FFEE33FE749C2F69
:103C7600F58274653EF583E493FE740193FFEF25A8
:103C860066F566EE3565F565E56BB40110900028BE
:103C9600E0FEA3E0FFEF4E7004056C8003756C0038
:103CA600E56CC394144008756C00A212B39212D34B
:103CB600E56B648094815003023F65C3E5696480C7
:103CC60094864003023D8B124D16E56B64047055D5
:103CD600AF69EF3395E0FE74102FF58274003EF560
:103CE60083E0256AF0AF69EF3395E0FE74102FF597
:103CF6008274003EF583E0FFEF3395E0FED3EF9547
:103D060066E5656480F8EE6480984016AF68AE6933
:103D1600EEFD3395E0FC74102DF58274003CF583BE
:103D2600EFF0124CC1E56B6402705AAF69EF339540
:103D3600E0FE74102FF58274003EF583E0FFC3EFBA
:103D4600956AFFEFF0AF69EF3395E0FE74102FF53B
:103D56008274003EF583E0FFEF3395E0FEC3EF95F6
:103D660068E5676480F8EE6480985016AF66AE69C1
:103D7600EEFD3395E0FC74102DF58274003CF5835E
:103D8600EFF0124CC1C3E569648094865003023E8D
:103D9600A774FA2569F569E56B64047072AF6AEF7A
:103DA600FD7C00AF69EF3395E0FEEF25E0FFEE33D3
:103DB600FE74222FF58274003EF583EC8DF0121E00
:103DC60048AF69EF3395E0FEEF25E0FFEE33FE7472
:103DD600222FF58274003EF583E0FEA3E0FFD3EFC9
:103DE6009566E5656480F8EE648098401FAF69EFDC
:103DF6003395E0FEEF25E0FFEE33FE74222FF582C9
:103E060074003EF583E567F0A3E568F0124DC5E55D
:103E16006B64026003023EA1AF69EF3395E0FEEFEB
:103E260025E0FFEE33FE74222FF58274003EF58303
:103E3600C083C082E0FEA3E0FFAD6A7C00C3EF9DB5
:103E4600FFEE9CFED082D083EEF0A3EFF0AF69EFD9
:103E56003395E0FEEF25E0FFEE33FE74222FF58268
:103E660074003EF583E0FEA3E0FFC3EF9568E567C7
:103E76006480F8EE648098501FAF69EF3395E0FEDA
:103E8600EF25E0FFEE33FE74222FF58274003EF537
:103E960083E565F0A3E566F0124DC574062569F560
:103EA60069900028E0FEA3E0FFEF4E705CE56BB47E
:103EB60005263014230569AF69D3EF6480949340D7
:103EC60003756900C214AF69EF3395E0FE90003EBA
:103ED600EEF0A3EFF0124DC5E56B64036003023FFD
:103EE6006530147B1569AF69C3EF64809480500315
:103EF600756913C214AF69EF3395E0FE90003EEE8C
:103F0600F0A3EFF0124DC58056E56BB405263014CC
:103F1600230569AF69D3EF64809492400375690005
:103F2600C214AF69EF3395E0FE90003EEEF0A3EFCA
:103F3600F0124DC5E56BB403263014231569AF693D
:103F4600C3EF648094805003756912C214AF69EFA1
:103F56003395E0FE90003EEEF0A3EFF0124DC5E57E
:103F66006BB40102D214E56B5406FFEF60109000AB
:103F76003EE0FEA3E0FFEF64094E7002C217900117
:103F8600E9E0FEA3E0FF900028E0FCA3E0FDED6F72
:103F96007002EC6E6002C217900028E0FEA3E0FFFC
:103FA6009001E9EEF0A3EFF030A302D21320A30AAA
:0A3FB600301307C213A217B39217CD
:013FC00022DE
:104CC100124E0E74A0124E267402124E269000103F
:104CD1007C03E0124DE7124E26A3DCF6E0124DE70D
:104CE100F5F0A3A3E0030354C045F0124E26900053
:104CF10014E0124DE7124E26C2B4124E01124E0EAE
:104D010074A0124E2674F0124E26A3E0124E26C253
:104D1100B4124E0122124E0E74A0124E26740212CB
:104D21004E26124E0E74A004124E26900010124E02
:104D31004B124DEFF0A3124E5E124E4B124DEFF09F
:104D4100A3124E5E124E4B124DEFF0A3124E5E12A5
:104D51004E4BFB543F124DEFF0A3124E5E124E4BE1
:104D6100FA541F124DEFF0EB23235403FD124E585A
:104D7100C2B4124E01124E0E74A0124E2674F012DD
:104D81004E26124E0E74A004124E26124E4BFB54A8
:104D910003C39D2405838007030201000302012B45
:104DA100A3F0F5F0124E58C2B4124E01124E0E7419
:104DB100A0124E2674F0124E26E5F0124E26C2B411
:104DC100124E01227AA07B807C1E900022124E9E00
:104DD100227AA07B80124E66ED900022F07AA0A389
:104DE1007C1D124ED32275F00A84C425F022C0E046
:0D4DF100C4540F75F00AA4F5F0D0E0540F83
:104DFE0025F02200D2B5000000D2B400000000223F
:104E0E00124E01C2B4000000C2B500000022D2B59D
:104E1E00000000C2B50000227E083392B4124E1C70
:104E2E00DEF833D2B40000A2B450040000A2B412D3
:104E3E004E1C400122C2B40000124E01227E08A276
:104E4E00B43300124E1CDEF7C322D2B4124E1C2213
:104E5E00C2B4124E1CD2B422124E0EEA124E26EBE1
:104E6E00124E26124E0EEA04124E26124E4BFD1212
:104E7E004E58C2B4124E0122124E0EEA124E26EBBC
:104E8E00124E26E6124E2608DCF9C2B4124E01224C
:104E9E00124E0EEA124E26EB124E26E0124E26A3AC
:104EAE00DCF9C2B4124E0122124E0EEA04124E2644
:104EBE008003124E5E124E4BF608DCF6124E58C2AE
:104ECE00B4124E0122124E0EEA04124E2680031226
:104EDE004E5E124E4BF0A3DCF6124E58C2B4124E7A
:024EEE0001229F
:1049E400202020202531642E2530326420253032C9
:1049F40062753A25303262753A253032627520206C
:104A0400202000202020202532642E2531642025FA
:104A1400303262753A25303262753A253032627529
:104A24002020202000253033642E253164202025C9
:104A34003032642E25316420415A2F454C312020D8
:104A44002000253033642E25316420202530326443
:104A54002E25316420415A2F454C32202020002538
:104A64003033642E2531642020253032642E2531E4
:104A7400642052412F4445432020200025303364D4
:104A84002E2531645720253032642E2531644E2082
:104A94004C4F2F4C412020200025303262752020BD
:104AA400202530326275202025303262753A253057
:104AB4003262753A2530326275202020200025307C
:104AC400352E31662020253032642E253164202095
:104AD400202020202025303264202000202B253067
:104AE40031642E2530316420202B253031642E256D
:104AF40030316420434F522020535450200025303D
:104B040033642E2531642020253032642E2531640F
:104B140020414E5420202531642E2531642000206C
:104B24002020204F20452035204A2046204C20209C
:104B3400202020002020202020202020454D45201A
:104B440020202020202020200020416E74656E6EDD
:104B54006120436F6E74726F6C6C6572200020204C
:104B640020202020207620362E31202020202020B6
:104B74002020002020204A414E4645424D415241CA
:104B840050524D41594A554E4A554C41554753454B
:104B9400504F43544E4F56444543004D4F4F4E20C3
:104BA4002053554E20202043415353494F435947E6
:104BB4004E55535341474954545441555255534CFF
:104BC400454F20202041515541522E52412F4445FA
:104BD40043415A2F454C32415A2F454C3100326DD6
:104BE4003A37303A32333A31333A36636D313047FB
:104BF40000205353492031306269742837323029F8
:104C040020202020202053534931316269742831F7
:104C1400383030292020202020205353493132625B
:104C24006974283336303029202020202020535323
:104C3400495F677261792834303936292020202071
:104C4400202041322D532D532031322062697420AB
:104C540020202020204D414232355F31306269747A
:104C64003130323420202020204D414232355F3112
:104C7400316269743230343820202020204D414282
:104C840032355F3132626974343039362020202065
:104C9400204D414232385F313262697434303936E2
:104CA4002020202020000F0C09010306171D664C4C
:0D4CB4000309030903090309560101020465
:10002E00E56B64016003125D4A200D0302060CC2EB
:10003E000D30120C900028E0FEA3E0FFEF4E601191
:10004E0090003EE0FEA3E0FFEF64134E600302015A
:10005E00E390003CE0FEA3E0FFC3EF9404EE648067
:10006E00948040030200FCAF1CAE1B12000EEF2466
:10007E0005FFEE3400FE7C007D0A121E128E748F78
:10008E00757B017A00796CC003C002C0017BFF7AD8
:10009E004979E49000DBEBF0A3EAF0A3E9F0AE744B
:1000AE00AF757C007D64121E129000DEEEF0A3EFA1
:1000BE00F0AE74AF757C007D64121E129000E0EC01
:1000CE00F0A3EDF0900012E0FF9000E2EFF0900050
:1000DE0011E0FF9000E3EFF0900010E0FF9000E4DD
:1000EE00EFF0D001D002D003123758020180AF1CBE
:1000FE00AE1B12000EEF2432FFEE3400FE7C007DAC
:10010E0064121E128E748F757B017A00796CC00397
:10011E00C002C0017BFF7A4A79079000DBEBF0A3A7
:10012E00EAF0A3E9F0AE74AF757C007D0A121E12E0
:10013E009000DEEEF0A3EFF0AE74AF757C007D0A9A
:10014E00121E129000E0ECF0A3EDF0900012E0FF12
:10015E009000E2EFF0900011E0FF9000E3EFF090DE
:10016E000010E0FF9000E4EFF0D001D002D00312B7
:10017E003758751500D3E515648094825042AF153B
:10018E0090003DE0FE75F003EEA4F58285F083E568
:10019E00822FF582E43583F583E58224E2F582E54C
:1001AE0083344BF583E493FFAE15EEFD3395E0FCFF
:1001BE00746C2DF58274003CF583EFF0051580B557
:1001CE00C3E51B64809480400302059C90006F740D
:1001DE002DF002059C90003EE0FEA3E0FFEF640AC6
:1001EE004E601190003EE0FEA3E0FFEF640B4E6008
:1001FE00030202877B017A00796CC003C002C00142
:10020E007BFF7A4A79299000DBEBF0A3EAF0A3E9B1
:10021E00F090002AE0FEA3E0FF7C007D0A121E1281
:10022E009000DEEEF0A3EFF090002AE0FEA3E0FFD8
:10023E007C007D0A121E129000E0ECF0A3EDF0900F
:10024E00002CE0FEA3E0FF7C007D0A121E1290003F
:10025E00E2EEF0A3EFF090002CE0FEA3E0FF7C00B6
:10026E007D0A121E129000E4ECF0A3EDF0D001D046
:10027E0002D00312375802059C90003EE0FEA3E028
:10028E00FFEF640C4E601190003EE0FEA3E0FFEF26
:10029E00640D4E600302032B7B017A00796CC00360
:1002AE00C002C0017BFF7A4A79469000DBEBF0A3D7
:1002BE00EAF0A3E9F090002EE0FEA3E0FF7C007DC3
:1002CE000A121E129000DEEEF0A3EFF090002EE068
:1002DE00FEA3E0FF7C007D0A121E129000E0ECF0FF
:1002EE00A3EDF0900030E0FEA3E0FF7C007D0A124B
:1002FE001E129000E2EEF0A3EFF0900030E0FEA3AD
:10030E00E0FF7C007D0A121E129000E4ECF0A3EDDB
:10031E00F0D001D002D00312375802059C90003E57
:10032E00E0FEA3E0FFEF640E4E601190003EE0FE93
:10033E00A3E0FFEF640F4E60030203F9900034E078
:10034E00FEA3E0FFEF247CF571EE34FCF570AF7187
:10035E00AE7012000E7C007D0A121E12C006C0077F
:10036E00AF71AE7012000E7C007D0A121E1290004C
:10037E00E4ECF0A3EDF0D007D0069000E2EEF0A38F
:10038E00EFF07B017A00796CC003C002C0017BFFE5
:10039E007A4A79639000DBEBF0A3EAF0A3E9F090E0
:1003AE000032E0FEA3E0FF7C007D0A121E129000D8
:1003BE00DEEEF0A3EFF0900032E0FEA3E0FF7C0053
:1003CE007D0A121E129000E0ECF0A3EDF0D001D0E9
:1003DE0002D003123758C3E5706480948040030244
:1003EE00059C900072742DF002059C90003EE0FE7C
:1003FE00A3E0FFEF64104E601190003EE0FEA3E01C
:10040E00FFEF64114E60030204F6900036E0FEA387
:10041E00E0FFEF24F8F573EE34F8F572900038E053
:10042E00FEA3E0FFEF247CF571EE34FCF570AF73A4
:10043E00AE7212000E7C007D0A121E12C006C0079C
:10044E00AF73AE7212000E7C007D0A121E12C00433
:10045E00C005AF71AE7012000E7C007D0A121E1226
:10046E00C006C007AF71AE7012000E7C007D0A127E
:10047E001E129000E4ECF0A3EDF0D007D006900031
:10048E00E2EEF0A3EFF0D005D0049000E0ECF0A384
:10049E00EDF0D007D0069000DEEEF0A3EFF07B017A
:1004AE007A00796CC003C002C0017BFF7A4A798062
:1004BE009000DBEBF0A3EAF0A3E9F0D001D002D07C
:1004CE0003123758C3E57264809480500690007111
:1004DE007445F0C3E57064809480400302059C90DF
:1004EE0000777453F002059C7B017A00796CC0038F
:1004FE00C002C0017BFF7A4A799D9000DBEBF0A32E
:10050E00EAF0A3E9F0900013E0FF9000DEEFF09028
:10051E000015E0FF9000DFEFF0900012E0FF90007A
:10052E00E0EFF0900011E0FF9000E1EFF09000108E
:10053E00E0FF9000E2EFF0D001D002D00312375866
:10054E00751500D3E515648094825042AF15900066
:10055E0014E0FE75F003EEA4F58285F083E5822F9C
:10056E00F582E43583F583E5822477F582E58334DD
:10057E004BF583E493FFAE15EEFD3395E0FC746E00
:10058E002DF58274003CF583EFF0051580B59000D3
:10059E0028E0FEA3E0FFC3EF9402EE648094805047
:1005AE003290003EE0FEA3E0FFC3EF940AEE6480BB
:1005BE009480401390003EE0FEA3E0FFD3EF941131
:1005CE00EE64809480400C90007E7444F090007F26
:1005DE007445F07F00125D5C751500D3E5156480DF
:1005EE009493501AAF15EF3395E0FE746C2FF5828D
:1005FE0074003EF583E0FF125D23051580DD200EAD
:10060E000302080CC20E90003EE0FEA3E0FFC3EF13
:10061E00940AEE64809480401590003EE0FEA3E0C4
:10062E00FFD3EF9411EE648094805002C2129001B9
:10063E00CAE0F8A3E0F9A3E0FAA3E0FB900004E01F
:10064E00FCA3E0FDA3E0FEA3E0FF1219AD126C02C5
:10065E007B007A00792078411218A47B007A007909
:10066E0000783F1217B3121B068E708F719001CA5D
:10067E00E0F8A3E0F9A3E0FAA3E0FB900068E0FC49
:10068E00A3E0FDA3E0FEA3E0FF1219AD126C027B06
:10069E00007A007900783F1217B3121B068E768F00
:1006AE00777B017A007984C003C002C0017BFF7A98
:1006BE004A79C29000DBEBF0A3EAF0A3E9F09001D7
:1006CE00CAE0F8A3E0F9A3E0FAA3E0FB90000CE087
:1006DE00FCA3E0FDA3E0FEA3E0FF1219AD9000DE47
:1006EE00121F5EAE70AF717C007D0A121E1290005A
:1006FE00E2EEF0A3EFF0AE70AF717C007D0A121E39
:10070E00129000E4ECF0A3EDF09000E6E576F0A395
:10071E00E577F0D001D002D0031237587F007E006B
:10072E007D007C00900004E0F8A3E0F9A3E0FAA3BA
:10073E00E0FB121A4A500690008A742DF0751500CF
:10074E00D3E515648094855042AF15900029E0FEE4
:10075E0075F006EEA4F58285F083E5822FF582E42E
:10076E003583F583E582249FF582E583344BF5834B
:10077E00E493FFAE15EEFD3395E0FC74902DF582FB
:10078E0074003CF583EFF0051580B5900028E0FE6F
:10079E00A3E0FFC3EF9402EE64809480400E9000BD
:1007AE00967420F09000977420F080217F007E00D8
:1007BE007D007C00900068E0F8A3E0F9A3E0FAA3C6
:1007CE00E0FB121A4A5006900095742DF0E56B640A
:1007DE0001602B7F40125D5C751500D3E5156480BA
:1007EE009493501AAF15EF3395E0FE74842FF58273
:1007FE0074003EF583E0FF125D23051580DD200FAA
:10080E0003020917C20F900022E0FEA3E0FFEF24BF
:10081E009CFFEE34FFFE12000E8E728F739000243A
:10082E00E0FEA3E0FFEF249CFFEE34FFFE12000E6D
:10083E008E708F717B017A00799CC003C002C0015B
:10084E007BFF7A4A79E09000DBEBF0A3EAF0A3E9B4
:10085E00F0AE72AF737C007D0A121E129000DEEEB7
:10086E00F0A3EFF0AE72AF737C007D0A121E1290F1
:10087E0000E0ECF0A3EDF0AE70AF717C007D0A12DB
:10088E001E129000E2EEF0A3EFF0AE70AF717C009E
:10089E007D0A121E129000E4ECF0A3EDF0D001D010
:1008AE0002D003123758900022E0FEA3E0FFC3EF00
:1008BE009464EE64809480500690009D742DF090A8
:1008CE000024E0FEA3E0FFC3EF9464EE6480948006
:1008DE0050069000A3742DF0E56B6401602B7F141D
:1008EE00125D5C751500D3E51564809493501AAFB4
:1008FE0015EF3395E0FE749C2FF58274003EF58360
:10090E00E0FF125D23051580DD201003020B19C2D6
:10091E0010900027E0FFEF904CBE93FFEF3395E071
:10092E00FEAC5BAD5C121E008E448F45AF42AE41F5
:10093E0012000E7C007D0A121E12C006C007AF42C6
:10094E00AE4112000E7C007D0A121E129000E4ECE5
:10095E00F0A3EDF0D007D0069000E2EEF0A3EFF09A
:10096E007B017A0079B4C003C002C0017BFF7A4BD1
:10097E0079029000DBEBF0A3EAF0A3E9F0AE46AF0C
:10098E00477C007D0A121E129000DEEEF0A3EFF0FF
:10099E00AE46AF477C007D0A121E129000E0ECF0CE
:1009AE00A3EDF0AE44AF457C007D0A121E129000FE
:1009BE00E6EEF0A3EFF0AE44AF457C007D0A121ECA
:1009CE00129000E8ECF0A3EDF0D001D002D00312AB
:1009DE003758C3E5416480948050069000BA742D58
:1009EE00F0A218B39218E508540CFFEFB4080820D3
:1009FE0018059000C4E4F0E508540CFFEFB40409A8
:100A0E002018069000C47401F0E508540CFFEFB4F2
:100A1E000C093017069000C4742AF0E5085403FF41
:100A2E00EFB402093018069000C37402F0E50854C2
:100A3E0003FFEFB401093018069000C37403F0E50C
:100A4E00085403FFEFB403093017069000C3742A4D
:100A5E00F090003EE0FEA3E0FFEF64124E60030252
:100A6E000AEE751500D3E515648094935042AF15C8
:100A7E0090003BE0FE75F014EEA4F58285F083E560
:100A8E00822FF582E43583F583E58224F5F582E540
:100A9E0083344BF583E493FFAE15EEFD3395E0FC06
:100AAE0074B42DF58274003CF583EFF0051580B516
:100ABE00AE44AF457C007D0A121E12EF2430FF902B
:100ACE0000C5EFF09000C6742EF0AE44AF457C002A
:100ADE007D0A121E12AF05EF2430FF9000C7EFF013
:100AEE007F54125D5C751500D3E5156480949350A8
:100AFE001AAF15EF3395E0FE74B42FF58274003EF5
:100B0E00F583E0FF125D23051580DDE56BB401145E
:100B1E0090003FE0FFEF904CAA93FF125D5C125DD8
:100B2E0041125D53301103020C7C7B017A00796C0B
:100B3E00C003C002C0017BFF7A4B79239000DBEB30
:100B4E00F0A3EAF0A3E9F0D001D002D00312375897
:100B5E007B017A007984C003C002C0017BFF7A4B0F
:100B6E0079389000DBEBF0A3EAF0A3E9F0D001D0E6
:100B7E0002D0031237587B017A00799CC003C00261
:100B8E00C0017BFF7A4B794D9000DBEBF0A3EAF0CE
:100B9E00A3E9F0D001D002D0031237587B017A00BE
:100BAE0079B4C003C002C0017BFF7A4B796290001A
:100BBE00DBEBF0A3EAF0A3E9F0D001D002D00312F0
:100BCE0037587F00125D5C751500D3E5156480946F
:100BDE0093501AAF15EF3395E0FE746C2FF58274B7
:100BEE00003EF583E0FF125D23051580DD7F401288
:100BFE005D5C751500D3E51564809493501AAF159E
:100C0E00EF3395E0FE74842FF58274003EF583E099
:100C1E00FF125D23051580DD7F14125D5C751500D6
:100C2E00D3E51564809493501AAF15EF3395E0FE1B
:100C3E00749C2FF58274003EF583E0FF125D230550
:100C4E001580DD7F54125D5C751500D3E51564804B
:100C5E009493501AAF15EF3395E0FE74B42FF582CE
:0F0C6E0074003EF583E0FF125D23051580DD2243
:106AF900014A00014800014900014300C117C116BC
:026B0900C115B4
:106BBE00752400D3E524648094A75004052480F343
:016BCE0022A4
:106BCF00752500D3E525648094935004052580F343
:016BDF002293
:106BE000752600D3E5266480949E5004052680F324
:016BF0002282
:106BF100752700D3E527648094855004052780F329
:016C01002270
:105EA000C290126BBE752D1F752C00E52CD3940784
:105EB0005011E52DC313F52DA2D79290126BBE059C
:105EC0002C80E8D290126BBED2927528037529E817
:105ED000752D00309110E52915297002152814FF41
:105EE000AE28EF4E70ED126BCF752C00E52CD394DD
:105EF000075013126BBEE52DC313F52D30910343EC
:105F00002D80052C80E6126BBEAF2D7E00EF752B29
:105F100000F52A7528037529E8752D00309110E5E4
:105F20002915297002152814FFAE28EF4E70ED12C6
:105F30006BCF752C00E52CD394075013126BBEE584
:105F40002DC313F52D309103432D80052C80E612CF
:105F50006BBEAF2D7E00EF252BF52BEE352AF52AF3
:105F6000C3E52A648094805006752A00752B00D3FF
:105F7000E52B940FE52A6480948E4006752A0E75F1
:105F80002B0FC29220B20DC3740F952BF52B740EFC
:085F9000952AF52AAE2AAF2B79
:015F980022E6
:10608900C294126BBE75331F753200E532D3940783
:106099005011E533C313F533A2D79294126BBE05A1
:1060A9003280E8D294126BBED296752E03752FE812
:1060B900753300309510E52F152F7002152E14FF3A
:1060C900AE2EEF4E70ED126BCF753200E532D394E0
:1060D900075013126BBEE533C313F53330950343F1
:1060E9003380053280E6126BBEAF337E00EF753127
:1060F90000F530752E03752FE8753300309510E5DE
:106109002F152F7002152E14FFAE2EEF4E70ED12C3
:106119006BCF753200E532D394075013126BBEE58D
:1061290033C313F533309503433380053280E612C8
:106139006BBEAF337E00EF2531F531EE3530F530EA
:10614900C3E530648094805006753000753100D302
:10615900E531940FE5306480948E400675300E75F4
:08616900310FC296AE30AF31D8
:01617100220B
:106B5700125EA08E468F47126089C374089FFF7428
:106B6700079EFE12000EC374849FF54274039EF5C0
:086B770041755B00755C012211
:1062EB00D290D294D291D295756100756200755D92
:1062FB0000755E00753400D3E53464809489504991
:10630B00126BE0C290C294126BE0C3E534648094CC
:10631B00895004D290D294E5622562F562E561352D
:10632B0061F561E55E255EF55EE55D355DF55D204C
:10633B0091080562E56270020561209508055EE52E
:10634B005E7002055D053480AEC290C294755B0031
:10635B00755C05AE61AF627C007D05121E008E463A
:10636B008F4720B20DC3740B9547F547740E9546B6
:10637B00F546C37468955EFF7401955DFE12000EC1
:10638B00C374B49FF55EE49EF55DAE5DAF5E7C00BD
:09639B007D05121E008E418F42A7
:0163A40022D6
:1063A500D290D294D291D295756100756200755DD7
:1063B50000755E00753500D3E5356480948A5049D3
:1063C500126BE0C290C294126BE0C3E53564809411
:1063D5008A5004D290D294E5622562F562E5613572
:1063E50061F561E55E255EF55EE55D355DF55D2092
:1063F50091080562E56270020561209508055EE574
:106405005E7002055D053580AEC290C294755B0075
:10641500755C02E56225E0F547E56133F54620B296
:106425000DC3740E9547F547740E9546F546C3742E
:1064350084955EFF7403955DFE12000EC374C29FC2
:10644500F55E74019EF55DE55E25E0F542E55D339B
:02645500F5410F
:016457002222
:10670700D290D294D291D295756100756200755D71
:1067170000755E00753600D3E5366480948B50496A
:10672700126BE0C290C294126BE0C3E536648094AA
:106737008B5004D290D294E5622562F562E561350B
:1067470061F561E55E255EF55EE55D355DF55D202C
:1067570091080562E56270020561209508055EE50E
:106767005E7002055D053680AEC290C294755B000F
:10677700755C0185614685624720B20DC3740F952C
:1067870047F547740E9546F546C37408955EFF7442
:1067970007955DFE12000EC374849FF54274039E35
:0267A700F541BA
:0167A90022CD
:1057BB00D292D291756100756200126BE09001ED8F
:1057CB00E4F09001EDE0FFD3EF6480948F5029D289
:1057DB0090126BE0C290126BE0E5622562F562E518
:1057EB00613561F5612091080562E5627002056122
:1057FB009001EDE004F080CAC290C292E562AE6106
:10580B007806CEC313CE13D8F9F5628E61AC61ADB9
:10581B0062E4121ACD7B007A00793478441218A412
:10582B007B007A00798078441219AD121B067C003C
:10583B007D05121E008E468F4720B20DC3740B954B
:10584B0047F547740E9546F546126BE0755B007590
:10585B005C05D296D295755D00755E00126BE0907B
:10586B0001EDE4F09001EDE0FFD3EF6480948F50F5
:10587B0029D294126BE0C294126BE0E55E255EF5C3
:10588B005EE55D355DF55D209508055EE55E7002B4
:10589B00055D9001EDE004F080CAC294C296E55E0E
:1058AB00AE5D7806CEC313CE13D8F9F55E8E5DC30D
:1058BB00E4955EFF7402955DFE12000EC3E49FFD3E
:1058CB0074019EFCEC121ACD7B007A00793478447B
:1058DB001218A47B007A00798078441219AD121B40
:0C58EB00067C007D05121E008E418F42DD
:0158F700228E
:1058F800D292D291756100756200126BE09001EE50
:10590800E4F09001EEE0FFD3EF6480948F5029D249
:1059180090126BE0C290126BE0E5622562F562E5D9
:10592800613561F5612091080562E56270020561E3
:105938009001EEE004F080CAC290C292E562AE61C6
:105948007805CEC313CE13D8F9F5628E61AC61AD7C
:1059580062E4121ACD7B007A0079E178441218A427
:105968007B007A00790078451219AD121B06EF25E5
:10597800E0F547EE33F54620B20DC3740E9547F5B2
:1059880047740E9546F546126BE0755B00755C0230
:10599800D296D295755D00755E00126BE09001EEAF
:1059A800E4F09001EEE0FFD3EF6480948F5029D2A9
:1059B80094126BE0C294126BE0E55E255EF55EE53D
:1059C8005D355DF55D209508055EE55E7002055D57
:1059D8009001EEE004F080CAC294C296E55EAE5D26
:1059E8007805CEC313CE13D8F9F55E8E5DC3E49562
:1059F8005EFF7404955DFE12000EC3E49FFD740201
:105A08009EFCEC121ACD7B007A0079E178441218DA
:105A1800A47B007A00790078451219AD121B06EFB5
:085A280025E0F542EE33F541E3
:015A30002253
:105A3100D292D291756100756200126BE09001EF14
:105A4100E4F09001EFE0FFD3EF6480948F5029D20E
:105A510090126BE0C290126BE0E5622562F562E59F
:105A6100613561F5612091080562E56270020561A9
:105A71009001EFE004F080CAC290C292E561C4F8DF
:105A810054F0C868F561E562C4540F48F562AC6131
:105A9100AD62E4121ACD7B007A0079617845121863
:105AA100A47B007A00798078451219AD121B068E0D
:105AB100468F4720B20DC3740F9547F547740E9575
:105AC10046F546126BE0755B00755C01D296D29586
:105AD100755D00755E00126BE09001EFE4F09001DE
:105AE100EFE0FFD3EF6480948F5029D294126BE0E2
:105AF100C294126BE0E55E255EF55EE55D355DF510
:105B01005D209508055EE55E7002055D9001EFE0A0
:105B110004F080CAC294C296E55DC4F854F0C86826
:105B2100F55DE55EC4540F48F55EC3E4955EFF7410
:105B310008955DFE12000EC3E49FFD74049EFCEC0B
:105B4100121ACD7B007A00796178451218A47B0086
:105B51007A00798078451219AD121B068E418F4269
:015B61002221
:1052C600D292D291756100756200126BF19001F075
:1052D600E4F09001F0E0FFD3EF6480948F5029D280
:1052E60090126BF1C290126BF1E5622562F562E5F0
:1052F600613561F5612091080562E562700205611C
:105306009001F0E004F080CAC290C292E561C4F850
:1053160054F0C868F561E562C4540F48F562D3E5F8
:10532600629552E5619551401885615785625885A9
:105336006151856252E56224FFF550E56134FFF55F
:105346004FC3E5629550E561954F501EE562240115
:10535600F558E5613400F55785614F856250E56281
:105366002401F552E5613400F551AC57AD58EC1205
:105376001ACD7B007A00796178451218A47B007AF1
:1053860000798078451219AD121B068E468F47208C
:10539600B20DC3740F9547F547740E9546F5461240
:1053A6006BF1755B00755C01D296D295755D0075E3
:1053B6005E00126BF19001F0E4F09001F0E0FFD393
:1053C600EF6480948F5029D294126BF1C294126BC1
:1053D600F1E55E255EF55EE55D355DF55D209508DA
:1053E600055EE55E7002055D9001F0E004F080CA9E
:1053F600C294C296E55DC4F854F0C868F55DE55EF2
:10540600C4540F48F55ED3E55E954EE55D954D4077
:1054160018855D55855E56855D4D855E4EE55E2437
:10542600FFF54CE55D34FFF54BC3E55E954CE55D58
:10543600954B501EE55E2401F556E55D3400F555A5
:10544600855D4B855E4CE55E2401F54EE55D3400D9
:10545600F54DC3E49556FF74089555FE12000EC32C
:10546600E49FFD74049EFCEC121ACD7B007A007951
:105476006178451218A47B007A0079807845121964
:08548600AD121B068E418F429E
:01548E0022FB
:105DA100D290D294D291D295756100756200755DE1
:105DB10000755E00753700D3E5376480948B5053CE
:105DC100C290C294753800D3E5386480948250043F
:105DD100053880F3C3E5376480948B5004D290D2A8
:105DE10094E5622562F562E5613561F561E55E255F
:105DF1005EF55EE55D355DF55D2091080562E56264
:105E010070020561209508055EE55E7002055D057D
:105E11003780A4C290C294755B00755C01AF62AE1D
:105E210061126BA68E618F62AF5EAE5D126BA68E44
:105E31005D8F5EAC61AD62E4121ACD7B007A0079B0
:105E41006178451218A47B007A007980784512198F
:105E5100AD121B068E468F4720B20DC3740F9547B6
:105E6100F547740E9546F546C3E4955EFF740895B3
:105E71005DFE12000EC3E49FFD74049EFCEC121A39
:105E8100CD7B007A00796178451218A47B007A00F5
:0E5E9100798078451219AD121B068E418F42A2
:015E9F0022E0
:1043890075080FE56424F8F554E56334F8F553E549
:104399004724F8F55AE54634F8F559C3E5536480DE
:1043A9009480500C74102554F554740E3553F553FC
:1043B900C3E55964809480500C7410255AF55A74D9
:1043C9000E3559F559900038E0FEA3E0FFC3EF948C
:1043D90084EE648094834025900022E0FEA3E0FFF0
:1043E900E5642FFFE5633EFEEF249CFFEE34FFFEFC
:1043F900C3EF9547F53AEE9546F5398023900022AB
:10440900E0FEA3E0FFE5542FFFE5533EFEEF249CB9
:10441900FFEE34FFFEC3EF955AF53AEE9559F5399B
:10442900D3E5609400E55F64809480402590002482
:10443900E0FEA3E0FFE5602FFFE55F3EFEEF249C71
:10444900FFEE34FFFEC3EF9542F53CEE9541F53B97
:10445900801B900024E0FEA3E0FFEF249CFFEE34D4
:10446900FFFEC3EF9542F53CEE9541F53B2017035E
:104479000246BBAE44AF457C007D02121E12D3E555
:104489003A9FEE6480F8E53964809840289001F1FC
:10449900E0FFEF20E506754A00754900054AAF4A75
:1044A900EFD394504003754A50E54AC3940A4054E7
:1044B90053080E804FAE44AF457C007D02121E1298
:1044C900C3E49FFFE49EFEC3E53A9FEE6480F8E5EE
:1044D9003964809850289001F1E0FFEF20E40675D7
:1044E9004A00754900054AAF4AEFD3945040037515
:1044F9004A50E54AC3940A400B53080D8006754A91
:1045090000754900AE44AF457C007D02121E12D3EE
:10451900E53C9FEE6480F8E53B6480984028900173
:10452900F1E0FFEF20E7067548007543000548AF45
:1045390048EFD394504003754850E548C3940A4066
:104549006153080B805CAE44AF457C007D02121EAE
:1045590012C3E49FFFE49EFEC3E53C9FEE6480F82E
:10456900E53B6480985035D3E5429400E541648089
:10457900948040289001F1E0FFEF20E6067548009D
:104589007543000548AF48EFD39450400375485030
:10459900E548C3940A400B5308078006754800751F
:1045A9004300AF3AAE3912000E8E3D8F3EC37428D8
:1045B900953EFFE4953DFEEF7802C333CE33CED866
:1045C900F9FFAD497C00C3EF9DF540EE9CF53FC373
:1045D900E53F648094805006753F00754000E54AC8
:1045E900C39450501DAF4A7E007C007D7F121E008F
:1045F9007C007D50121E12EF2480FFEF64FFF5FA54
:104609008027C3E53E9428E53D648094805017E5F2
:1046190049C394A050100549C3E53F648094804084
:10462900088540FA800375FA00AF3CAE3B12000ED4
:104639008E3D8F3EC37428953EFFE4953DFEEF788D
:1046490002C333CE33CED8F9FFAD437C00C3EF9D0F
:10465900F540EE9CF53FC3E53F64809480500675B4
:104669003F00754000E548C39450501DAF487E0097
:104679007C007D7F121E007C007D50121E12EF24EB
:1046890080FFEF64FFF5FE803BC3E53E9428E53DDE
:10469900648094805017E543C394A050100543C328
:1046A900E53F64809480401C8540FE801775FE00BC
:1046B9008012754A0075490075480075430075FAFE
:1046C9000075FE00E508C454F0FFEF240FFF9001C8
:0A46D900F1EFF09001F1E0FF8FA077
:0146E30022B4
:106B1F004310000043D8000044A2000045110000BC
:106B2F0045B400004622000000C700C70002000A5B
:106B3F000E0F03840E0F03840001000100000000FC
:086B4F0000000000000000003E
:106B0B00011400011663011200011700011A00C1E4
:036B1B000CC18B1F
:0300030002617225
:10617200C0E0C083C08263A201C083C082C0D07568
:10618200D000C006C007200B4F200C4CD2B330B356
:10619200020512051AAF1AC3EF64809488401CAF3F
:1061A20017EF3395E0FE74402FF58274003EF583BD
:1061B200E512F07512000517751A00E5122512F5A1
:1061C20012C3E51764809484404F751700D20C9077
:1061D2000048E0FF8F128041200B3E300C3BE5125D
:1061E2002512F512A2D792B3051AAF1AC3EF648033
:1061F2009488401A0517AF17EF3395E0FE74482FC5
:10620200F58274003EF583E0FF8F12751A00C3E534
:1062120017648094A04002D20BD007D006D0D0D011
:0D62220082D08363A201D082D083D0E0320D
:104EF000900048E563F0A3E564F0E5602484FFE5F5
:104F00005F3403FE90004AEEF0A3EFF090004CE512
:104F100046F0A3E547F0E5422484FFE5413403FE73
:104F200090004EEEF0A3EFF0E50B2484FFE50A3489
:104F300003FE900050EEF0A3EFF0900022E0FEA3FD
:104F4000E0FF900052EEF0A3EFF0900024E0FEA30B
:104F5000E0FF900054EEF0A3EFF0900028E0FEA3F5
:104F6000E0FF900056EEF0A3EFF0900058E544F01B
:104F7000A3E545F030170B90005AE4F0A37401F05C
:104F8000800890005AE4F0A3E4F0900015E0FFEFF1
:104F90003395E0FE90005CEEF0A3EFF0900014E09B
:104FA000FFEF3395E0FE90005EEEF0A3EFF090008F
:104FB00013E0FFEF3395E0FE900060EEF0A3EFF01A
:104FC000900012E0FFEF3395E0FE900062EEF0A358
:104FD000EFF0900011E0FFEF3395E0FE900064EEFB
:104FE000F0A3EFF0900041E0F516900040E4F0A34C
:104FF0007463F0C3E5166480948840030250D5C3FF
:10500000E5166480948050030250D5900042E0F58C
:1050100018A3E0F519AF16EF3395E0FEEF25E0FF9A
:10502000EE33FE74372FF582746B3EF583E493FE06
:10503000740193FFD3E5199FEE6480F8E51864804E
:10504000984021AF16EF3395E0FEEF25E0FFEE33F9
:10505000FE74372FF582746B3EF583E493F5187474
:105060000193F519AF16EF3395E0FEEF25E0FFEE63
:1050700033FE74472FF582746B3EF583E493FE7420
:105080000193FFC3E5199FEE6480F8E518648098EA
:105090005021AF16EF3395E0FEEF25E0FFEE33FE33
:1050A00074472FF582746B3EF583E493F518740111
:1050B00093F519AF16EF3395E0FEEF25E0FFEE33E1
:1050C000FE74222FF58274003EF583E518F0A3E507
:1050D00019F0124DC5E516B40805A217B3921722B0
:03002B0002622F3F
:10622F00C0E0C0F0C083C08263A201C083C082C03F
:10623F00D075D000C000C001C002C003C004C005AB
:10624F00C006C007C2CF75A61E75A6E11509AF0916
:10625F00EF706775090490003AE0FEA3E0FFEF8E40
:10626F00F0121FE1629B000062A0000162A5000214
:10627F0062AA000362AF000462B4000562B90006AF
:10628F0062BE000762C30008000062C61262EB80A4
:10629F00261263A58021126707801C125DA180174B
:1062AF00126B5780121257BB800D1258F8800812CC
:1062BF005A3180031252C6124389D007D006D00537
:1062CF00D004D003D002D001D000D0D0D082D08360
:0C62DF0063A201D082D083D0F0D0E03266
:030023000269EF80
:1069EF00C0E0C0F0C083C08263A201C083C082C078
:1069FF00D075D000C000C001C002C003C004C005E4
:106A0F00C006C007C2AC30981AC298E599B43F03CC
:106A1F001250E0E599B4210B12548FD20DD20ED241
:106A2F000FD210C299D2ACD007D006D005D004D067
:106A3F0003D002D001D000D0D0D082D08363A20186
:096A4F00D082D083D0F0D0E032F7
:03000B0002645834
:10645800C0E0C0F0C083C08263A201C083C082C014
:10646800D075D000C000C001C002C003C004C00580
:10647800C006C007758A00758C4C75A61E75A6E106
:106488000514AF14C3EF6480948A4016300B13755B
:106498001400751700751A00C20CC20B7512001291
:1064A8004EF0E51375F007121D86AFF0EF701E125F
:1064B8003B76301104D20DD210E56B600730110421
:1064C800D20ED20F12002E124D16124DD21513AF46
:1064D80013EF700C75134ED211301104D20ED20F77
:1064E800D007D006D005D004D003D002D001D00008
:1064F800D0D0D082D08363A201D082D083D0F0D014
:02650800E0327F
:10217B00758FFF758921758DFF438780759850D2B8
:10218B008CD28ED2CA75CB4C75CA0043B81143B7EB
:10219B0021D28875D90243D84075DA4275DE42C226
:1021AB00117513467509017F02125CEB125D3875D0
:1021BB006C00900040E4F0A37463F020A00312695C
:1021CB007575A8B275A707E56B70FC900036E0FC3F
:1021DB00A3E0FDEC121ACD7B007A00792078411236
:1021EB0019AD7B007A00793478C31217B39001CA0A
:1021FB00E0F8A3E0F9A3E0FAA3E0FB1218A4900027
:10220B001E121F5E900038E0FCA3E0FDEC121ACD0D
:10221B007B007A00792078411219AD7B007A007926
:10222B00B478C21217B39001CAE0F8A3E0F9A3E0A7
:10223B00FAA3E0FB1218A490001A121F5E90001173
:10224B00E0FCEC121AD27B007A0079B478441219B4
:10225B00ADC004C005C006C007900012E0FCEC1234
:10226B001AD27B007A0079C078411219ADA804A963
:10227B0005AA06AB07D007D006D005D0041217B3BA
:10228B00C004C005C006C007900010E0FCEC121A99
:10229B00D27B007AC079A878471219ADA804A9059A
:1022AB00AA06AB07D007D006D005D0041217B390FF
:1022BB000044121F5E900014E0FFEF3395E0FEFD2B
:1022CB00FCEF2409FFEE3400FEED3400FDEC34008E
:1022DB00FC7B0C7A0079007800126A58A804A905D7
:1022EB00AA06AB07900015E0FFEF3395E0FEFDFC6F
:1022FB00EF24D0FFEE3407FEED3400FDEC3400FC90
:10230B00EB2FFFEA3EFEE93DFDE83CFC7B077A0044
:10231B0079007800121E5E7B047A00790078001237
:10232B006A58C004C005C006C007900015E0FFEF57
:10233B003395E0FEFDFC7B6F7A0179007800121E6D
:10234B005ED003D002D001D000C3EF9BFFEE9AFE0C
:10235B00ED99FDEC98FCC004C005C006C0079000C9
:10236B0014E0FFEF3395E0FEFDFC7B137A0179005F
:10237B007800121E5E7B097A0079007800126A5889
:10238B00A804A905AA06AB07D007D006D005D00430
:10239B00EB2FFBEA3EFAE93DF9E83CF8900013E03D
:1023AB00FFEF3395E0FEFDFCEB2FFFEA3EFEE93D30
:1023BB00FDE83CFCEF247AF511EE34E0F510ED343A
:1023CB0000F50FEC3400F50E900028E0FEA3E0FFC3
:1023DB00EF64014E70487B017A007908C003C0029C
:1023EB00C0017B017A007968900193EBF0A3EAF0CE
:1023FB00A3E9F0AF11AE10AD0FAC0E900196121F0A
:10240B005E900044E0FCA3E0FDA3E0FEA3E0FF90A0
:10241B00019A121F5ED001D002D003123FC190006F
:10242B0028E0FEA3E0FFEF4E60030226007B017A5B
:10243B00007908C003C002C0017B017A0079689063
:10244B00010BEBF0A3EAF0A3E9F0AF11AE10AD0F67
:10245B00AC0E90010E121F5E900044E0FCA3E0FD59
:10246B00A3E0FEA3E0FF900112121F5ED001D00289
:10247B00D0031229D590001AE0FCA3E0FDA3E0FEE7
:10248B00A3E0FF12567B7B547AE379457840121810
:10249B00A4C004C005C006C007900016E0FCA3E072
:1024AB00FDA3E0FEA3E0FF125691A804A905AA061E
:1024BB00AB07D007D006D005D0041218A4C004C0B7
:1024CB0005C006C007900068E0FCA3E0FDA3E0FE9A
:1024DB00A3E0FF12567BA804A905AA06AB07D007F9
:1024EB00D006D005D0041218A4C004C005C006C085
:1024FB0007AF11AE10AD0FAC0EC004C005C006C0C7
:10250B00077FAB7EAA7D2A7C3C900044E0F8A3E0D9
:10251B00F9A3E0FAA3E0FB1217B3900146121F5E7A
:10252B00D007D006D005D004120C7DC004C005C066
:10253B0006C007AF11AE10AD0FAC0EC004C005C086
:10254B0006C0077FAB7EAA7D2A7CBC900044E0F8D6
:10255B00A3E0F9A3E0FAA3E0FB1217B39001461234
:10256B001F5ED007D006D005D004120C7DD003D04F
:10257B0002D001D0001217AF7B007A007987784325
:10258B001219ADA804A905AA06AB07D007D006D02F
:10259B0005D0041217B37B007A00797A78441218AD
:1025AB00A4121B068E0C8F0DAC0CAD0DEC121ACDBC
:1025BB00C004C005C006C00790003CE0FEA3E0FFCE
:1025CB00EF7802C333CE33CED8F9FF741F2FF582C9
:1025DB00746B3EF583121F2ED007D006D005D004A6
:1025EB001218A47B007A00797A78441219AD121B69
:1025FB00068E1B8F1C900028E0FEA3E0FFEF640209
:10260B004E7014900068121F6A3F82D0E59000084C
:10261B00121F6A40C39DB2900028E0FEA3E0FFEFBB
:10262B0064034E7014900068121F6A3F3566CF909A
:10263B000008121F6A40A73B64900028E0FEA3E04D
:10264B00FFEF64044E7014900068121F6ABF018F75
:10265B00C5900008121F6A40953F7D900028E0FE50
:10266B00A3E0FFEF64054E7014900068121F6A3EE2
:10267B00C44D01900008121F6A3FB91687900028BD
:10268B00E0FEA3E0FFEF64064E7014900068121F8B
:10269B006A3F32B6AE900008121F6A401F2B0290A1
:1026AB000028E0FEA3E0FFEF64074E701490006873
:1026BB00121F6A00000000900008121F6A40BC7ACB
:1026CB00E1900028E0FEA3E0FFEF64084E706790F6
:1026DB000032E0FCA3E0FDEC121ACD7B007A00790E
:1026EB002078411219AD9001CAE0F8A3E0F9A3E0FC
:1026FB00FAA3E0FB1218A4900008121F5E9000349E
:10270B00E0FCA3E0FDEC121ACD7B007A0079207877
:10271B00411219AD7B007A0079B478C21217B390CD
:10272B0001CAE0F8A3E0F9A3E0FAA3E0FB1218A4B6
:10273B00900068121F5E900028E0FEA3E0FFC3EF3D
:10274B009409EE648094804003022854900044E086
:10275B00FCA3E0FDA3E0FEA3E0FFC004C005C006A0
:10276B00C007AF11AE10AD0FAC0E9001B6121F5ECD
:10277B00D007D006D005D0041246E4900170121F8A
:10278B005E7B017A00790CC003C002C0017B017A29
:10279B0000790090016DEBF0A3EAF0A3E9F0900053
:1027AB0008E0FCA3E0FDA3E0FEA3E0FF90017412A0
:1027BB001F5E900068E0FCA3E0FDA3E0FEA3E0FF3A
:1027CB00900178121F5ED001D002D0031231DC9041
:1027DB000028E0FEA3E0FFEF4E705A900000E0FCF3
:1027EB00A3E0FDA3E0FEA3E0FF12567B7B007A5033
:1027FB0079C778451218A4C004C005C006C007905D
:10280B0000D0121F6A48B98C00D007D006D005D073
:10281B0004126847A804A905AA06AB07900000E0BC
:10282B00FCA3E0FDA3E0FEA3E0FF1217AF900004B2
:10283B00121F5E8014900000E0FCA3E0FDA3E0FEFD
:10284B00A3E0FF900004121F5E900028E0FEA3E0BF
:10285B00FFEF64094E705C90002EE0FCA3E0FDECF2
:10286B00121ACD7B007A00792078411219AD9001B4
:10287B00CAE0F8A3E0F9A3E0FAA3E0FB1218A490D6
:10288B00000C121F5E900030E0FCA3E0FDEC121A6E
:10289B00CD7B007A00792078411219AD9001CAE006
:1028AB00F8A3E0F9A3E0FAA3E0FB1218A49000044C
:1028BB00121F5E900028E0FEA3E0FFEF640A4E704B
:1028CB005C90002AE0FCA3E0FDEC121ACD7B007AB1
:1028DB0000792078411219AD9001CAE0F8A3E0F914
:1028EB00A3E0FAA3E0FB1218A490000C121F5E9059
:1028FB00002CE0FCA3E0FDEC121ACD7B007A0079F2
:10290B002078411219AD9001CAE0F8A3E0F9A3E0D9
:10291B00FAA3E0FB1218A4900004121F5E9001CAE8
:10292B00E0F8A3E0F9A3E0FAA3E0FB90000CE0FCD5
:10293B00A3E0FDA3E0FEA3E0FF1219AD7BCD7ACCA3
:10294B00794C783D1217B37B007A007920784112CD
:10295B0018A4121B068E638F649001CAE0F8A3E0E3
:10296B00F9A3E0FAA3E0FB900004E0FCA3E0FDA3D5
:10297B00E0FEA3E0FF1219AD7BCD7ACC794C783D0C
:10298B001217B37B007A00792078411218A4121B1E
:10299B00068E5F8F607F007E007D207C41900068FB
:1029AB00E0F8A3E0F9A3E0FAA3E0FB1218A490016E
:1029BB00CAE0F8A3E0F9A3E0FAA3E0FB1219AD1209
:0A29CB001B068E0A8F0B0221D22298
:105C8400EFC0E0C283740F125CB97430125CC37449
:105C940005125CB97430125CC37401125CB97430BF
:105CA400125CC37401125CB9D0E01460027408443D
:105CB40020125CD1227D000000DDFCD5E0F72254E7
:105CC400F053800F4280C282D283C28322C2828078
:105CD40002D282C0E0125CDFD0E0C454F053800FE3
:105CE4004280D283C28322125C84125D1D74061228
:105CF4005CD1125D1D740E125CD1125D1D74011213
:105D04005CD1125D1D7440125CD1125D6A125D1D7E
:105D14007480125CD1125D4A22740A125CB922EFBB
:105D2400C0E0125D1DD0E0125CD522125D1D74022C
:105D3400125CD122125D1D7401125CD122125D1D10
:105D4400740E125CD122125D1D740C125CD12212ED
:105D54005D1D740F125CD122EFC0E0125D1DD0E016
:105D64004480125CD122905D797E28E493FF125D19
:105D740023A3DEF7220004040E0E1F1F00001F1FC2
:105D84000E0E04040000101C1F1C1000000001076C
:0D5D94001F070100000E11171917110E0056
:106BA6007A107B00EE6BFB8BF053F080ABF033EF8B
:086BB60033FFEE33FEDAEE229C
:1068E4009001EBEEF0A3EFF09001EBE0FEA3E0FFEC
:1068F4007C037DE8121E12EF2430F5993099FDC215
:10690400999001EBE0FEA3E0FF7C037DE8121E12E8
:106914007E007F64CFCDCFCECCCE121E12EF2430BA
:10692400F5993099FDC2999001EBE0FEA3E0FF7C5C
:10693400007D64121E127E007F0ACFCDCFCECCCE56
:10694400121E12EF2430F5993099FDC2999001EB93
:10695400E0FEA3E0FF7C007D0A121E12AF05EF24C7
:1069640030F5993099FDC2997599003099FDC29915
:016974002200
:1050E0009001E1121F6A000186A020983E9001E124
:1050F000E0FCA3E0FDA3E0FEA3E0FFEC4D4E4F601B
:105100002A9001E1E0FCA3E0FDA3E0FEA3E0FF7B29
:10511000FF7AFF79FF78FFEF2BFFEE3AFEED39FDC6
:10512000EC38FC9001E1121F5E80BFC298AF99EF8E
:10513000121FBB518561519162519D6351A564510C
:10514000B16551BD6651C96751D56851E16951EDED
:105150006A51F96B52056C52116D521D6E522B6FD4
:10516000523370524171524972525773525F7452A6
:105170007275528076528E77529C7852AA7952B8C4
:105180007A000052C5900022E0FEA3E0FF1268E41E
:1051900022900024E0FEA3E0FF1268E422AF45AEB7
:1051A000441268E422900028E0FEA3E0FF1268E4C5
:1051B0002290002AE0FEA3E0FF1268E42290002C77
:1051C000E0FEA3E0FF1268E42290002EE0FEA3E0E0
:1051D000FF1268E422900030E0FEA3E0FF1268E4D2
:1051E00022900032E0FEA3E0FF1268E42290003437
:1051F000E0FEA3E0FF1268E422900036E0FEA3E0A8
:10520000FF1268E422900038E0FEA3E0FF1268E499
:105210002290003AE0FEA3E0FF1268E422E50D24AC
:1052200088FFE50C3413FE1268E422AF47AE461245
:1052300068E422E5422484FFE5413403FE1268E479
:1052400022AF64AE631268E422E5602484FFE55F68
:105250003403FE1268E422AF0BAE0A1268E4223077
:1052600017087F017E001268E4227F007E0012682A
:10527000E422900010E0FFEF3395E0FE1268E42294
:10528000900011E0FFEF3395E0FE1268E4229000F9
:1052900012E0FFEF3395E0FE1268E422900013E085
:1052A000FFEF3395E0FE1268E422900014E0FFEF78
:1052B0003395E0FE1268E422900015E0FFEF33958D
:0552C000E0FE1268E4AD
:0152C50022C6
:106662009001D6E4F0A3E4F09001DCE4F09001DCC8
:10667200E0FFD3EF6480948340030266FE9001D86A
:10668200121F6A000186A020983E9001D8E0FCA368
:10669200E0FDA3E0FEA3E0FFEC4D4E4F602A900127
:1066A200D8E0FCA3E0FDA3E0FEA3E0FF7BFF7AFFBE
:1066B20079FF78FFEF2BFFEE3AFEED39FDEC38FC67
:1066C2009001D8121F5E80BFC2989001D6E0FEA34F
:1066D200E0FF7C007D0A121E00AD997C00EF2DFFC9
:1066E200EE3CFEEF24D0FFEE34FFFE9001D6EEF03A
:1066F200A3EFF09001DCE004F002666F9001D6E0B7
:04670200FEA3E0FF13
:016706002270
:10548F009001E5121F6A000186A020983E9001E569
:10549F00E0FCA3E0FDA3E0FEA3E0FFEC4D4E4F6068
:1054AF002A9001E5E0FCA3E0FDA3E0FEA3E0FF7B73
:1054BF00FF7AFF79FF78FFEF2BFFEE3AFEED39FD14
:1054CF00EC38FC9001E5121F5E80BFC298AF99EFD8
:1054DF00121FBB552261553162554063554F6455BC
:1054EF005E65556D66557C67558B68559A6955A9EC
:1054FF006A55B86B55C76C55D66D55E57455EB7538
:10550F0055F776560377560F78561B7956277A003C
:10551F00005632126662900022EEF0A3EFF0124DA9
:10552F00C522126662900024EEF0A3EFF0124DC573
:10553F0022126662900026EEF0A3EFF0124DC52204
:10554F00126662900028EEF0A3EFF0124DC5221202
:10555F00666290002AEEF0A3EFF0124DC52212669C
:10556F006290002CEEF0A3EFF0124DC5221266628E
:10557F0090002EEEF0A3EFF0124DC522126662904E
:10558F000030EEF0A3EFF0124DC5221266629000CC
:10559F0032EEF0A3EFF0124DC52212666290003486
:1055AF00EEF0A3EFF0124DC522126662900036EEB8
:1055BF00F0A3EFF0124DC522126662900038EEF0A4
:1055CF00A3EFF0124DC52212666290003AEEF0A3DF
:1055DF00EFF0124DC522A217B392172212666290F6
:1055EF000010EFF0124CC122126662900011EFF022
:1055FF00124CC122126662900012EFF0124CC122BF
:10560F00126662900013EFF0124CC1221266629084
:10561F000014EFF0124CC122126662900015EFF0E9
:03562F00124CC159
:015632002255
:1017AC00021B72E86480F8E933E83360110460F0DE
:1017BC00ED33EC337009E8FCE9FDEAFEEBFF2204A3
:1017CC0060DED3EB9FEA9EE99DE8C2E78CF0C2F79E
:1017DC0095F0400CE8CCF8E9CDF9EACEFAEBCFFB6A
:1017EC00121B3D85D0F05804700320D5B3E804706B
:1017FC00075002B2D5021B7C92D5EC0460F7E4CC06
:10180C00C0E0C398F8603B94186008400DD0E0FB32
:10181C00021B54E4FBFAC9FC8028E830E406E4C956
:10182C00FBE4CAFCE830E305E4C9CACBFCE8540786
:10183C006010F8C3E913F9EA13FAEB13FBEC13FC91
:10184C00D8F130F52FC3E49CFCEF9BFFEE9AFEED34
:10185C0099FDD0E0FBEF4E4D4C701222DB03021BC6
:10186C0079EC2CFCEF33FFEE33FEED33FDED30E77E
:10187C00EB021B54EF2BFFEE3AFEED39FDD0E0FBF3
:10188C0050130BBB0003021B7CED13FDEE13FEEF9C
:08189C0013FFEC13FC021B54C6
:1018A400EC4D6011E8497017ED33EC3304600DE43E
:1018B400FCFFFEFD22E933E8330470F8021B7212C8
:1018C4001B3D58046009E4CC2481500628500902C9
:1018D4001B7C284003021B79C0E0EB4A7044B980AA
:1018E40006D0E0FB021B68EF4E701CBD8008EBFFC6
:1018F400EAFEE9FD80EBE98DF0A4FEE5F002198D26
:10190400E9CDF9EAFEEBFFEF89F0A4FCE5F0CE891E
:10191400F0A42EFFE435F0CD89F0A42DFEE435F0DB
:101924008067EF4E7005BD80D780C3EF8BF0A4AC09
:10193400F0EE8BF0A42CFCE435F0F8EF8AF0A42C44
:10194400E5F038FCE433CB8DF0A42CFCE5F03BF857
:10195400EE8AF0A42CFCE5F038F8E433CF89F0A447
:101964002CFCE5F038CF3400CE89F0A42FFFE5F04D
:101974003EFEE433C98DF0A42EFEE5F039CD8AF0A5
:10198400A42FFFE5F03EFEE43DFD33D0E0FB50071D
:101994000BBB000F021B7CEC2CFCEF33FFEE33FE81
:0619A400ED33FD021B54AF
:1019AA00021B7CEC5D046005E859047003021B729B
:1019BA00121B3D580460F6EC4860F2EC7004FDFE20
:1019CA00FF22C860DB2481C85009C3986002500610
:1019DA00021B799850CAF582E9294B4A7005AB82F5
:1019EA00021B6875F0007C1A7880C3EF9BEE9AEDB3
:1019FA0099400DC3EF9BFFEE9AFEED99FDE842F088
:101A0A00DC23ACF0D0E0FFD0E0FED0E0FDAB8220DA
:101A1A00E7101BEB60BAEC2CFCEF33FFEE33FEED64
:101A2A0033FD021B54E803F830E705C0F075F000F7
:101A3A00EF2FFFEE33FEED33FD40B830E7C280AA48
:101A4A0074F8CC6480CCC86480C8F582046043C34F
:101A5A00EB9FF5F0EA9E42F0E99D42F0E89C45F0E2
:101A6A0060305018E5825FFFE582F42B5582FB5007
:101A7A00210ABA001D09B90019088016E5825BFB24
:101A8A00E582F42F5582FF50090EBE00050DBD00F8
:101A9A00010CC3EB9FF5F0EA9E42F0E99D42F0E8A3
:0D1AAA009C45F06007CC4820E701B3EC221A
:101AB700ED33EC33600A047003BD8004ECB2E7FC3D
:011AC70022FC
:101AC80075F020800E75F010800575F0087D007E99
:101AD800007F003392D530D503121EADEC33401091
:101AE800EF33FFEE33FEED33FDEC33FCD5F0ED22A2
:0E1AF800E5F0247EA2D513CC92E7CDCEFF22DE
:101B0600EDD2E7CD33EC3392D524814006E4FFFED7
:101B1600FDFC22FCE4CFCECDCC24E0501174FF8036
:101B2600EDC3CC13CCCD13CDCE13CECF13CF0470D3
:071B3600F030D5DE021EAD08
:1036F300E57824DBF582E43400F583E00578229055
:1037030000D83009039000DBE475F001121F9B021F
:103713001DA82002E97F2ED2028018EF540F2490B7
:10372300D43440D4FF30060BEF24BFB41A00500347
:103733002461FFE57960021579057CE57C7002055B
:103743007B30090E9000D8E475F001121F9BEF0245
:103753001DEE026B7F7403D2098003E4C209F5787E
:103763009000D8121FB2E4F579F57BF57CE579601A
:10377300077F2012373680F5757AFFC203C202C273
:1037830004C205C207C208C20A123702FF700D3015
:1037930009057F00123747AF7CAE7B22B4255FC299
:1037A300D5C206123702FF24D0B40A00501A75F0AE
:1037B3000A787930D50508B6FF0106C6A426F62097
:1037C300D5047002D20580D924CFB41A00EF500477
:1037D300C2E5D206023A39D20380C6D20280C0D2F1
:1037E3000480BCD2D580BAD20780B47F201237368A
:1037F3002004077401B5790040F11236F3FF123744
:1038030036023770D20AD20880951236F3FB12368D
:10381300F3FA1236F3F94A4B700679377A3B7BFF9A
:1038230020042EE579602A7E008E82758300121DA6
:10383300C160060EEE657A70F0C2D5EBC0E0EAC057
:10384300E0E9C0E0EE123A9AD0E0F9D0E0FAD0E035
:10385300FB121DA8FF60AAEBC0E0EAC0E0E9C0E0EC
:10386300123736D0E02401F9D0E03400FAD0E0FB7F
:10387300E57A0460DCD57AD98087D20480A2123A33
:103883007C60F7E57A700104121B87A97A600DE565
:103893007A600914F57A123B24EF60F3EA30E70209
:1038A300F404C3995079EAF4257A0430E701E40477
:1038B300F57A800D123A7C60C1EA057A257A121BEB
:1038C30087EA900107F030E701E4257A04D57A040A
:1038D30020070114123A9AE4C0E0123B2490010736
:1038E300E0601320E70714F012371E802204F0D0A3
:1038F300E014C0E07F0012371EE57A600712371527
:10390300157A800B300703123715D0E0023770D0D9
:10391300E00480C4123A7C609EE57A04121B87900F
:103923000107EAF0E57A2007026001042404123A51
:013933009AF9
:1039340074FF04C0E0123B2412371EE57A2007020C
:103944006003123715D0E0B57AE87F451237289026
:103954000107E07F2B30E7047F2DF404C0E0123729
:1039640036D0E075F00A84C0F012371FD0E0123769
:103974001F023770791080027908C208C20A8008D1
:10398400D2D5790A8004790AC2D5E57A047002F5A1
:103994007AE4FAFDFEFF1236F3FC7B0820031312CF
:1039A40036F3FD7B1030020A1236F3FE1236F3FFB3
:1039B4007B20EC3382D592D55013C3E43002069FAA
:1039C400FFE49EFEE42003039DFDE49CFCE4CBF8AD
:1039D400C203EC700CCFCECDCCE824F8F870F380A1
:1039E40017C3EF33FFEE33FEED33FDEC33FCEB3363
:1039F400FB994002FB0FD8E9EB300305F8D0E0C493
:103A040048B203C0E00AEC4D4E4F78207B0070C2F0
:103A1400EAB57A0040BCC0E0123A9CD0F0D0E02075
:103A24000304C4C0E0C4B203C0F012371FD0F0D501
:103A3400F0EB023770121FBB380D5339785837DE5C
:103A44004C37DA42397C4F39844439844937F3435B
:103A5400398A5538B7463917453881473B57503767
:103A6400E22D37E62E38092B37EA233807203B406E
:103A74002A37A24800003801E57AB4FF03757A06B4
:103A84001236F3FC1236F3FD1236F3FE1236F3FF50
:103A9400900100021BC4790AA2D52005143007093D
:103AA400B910020404B9080104A2D5200802500187
:103AB400042004689204B579005034C0E07F2030BB
:103AC40005197F30A20472087207500F123AF3C22C
:103AD40004C208C207C20A7F30800F300703E9C05E
:103AE400E0123736300703D0E0F9D0E0B579CC30B6
:103AF40007177F30B9100C1237367F583006077F0E
:103B0400788003B908031237363004057F2D023755
:103B1400367F20200AF87F2B2008F322920480CFDE
:103B24007F00B40700500B2400F582E43401F583D0
:103B3400E0FF22286E756C6C2900D2031236F33034
:103B440003F8C203787930D50108F60237A22D5064
:103B54004349581236F32403B405004001E4903B72
:103B64005293123727743A123727D2057579040213
:023B740039789E
:0D6C0200ED33EC3360065004EC6480FC229E
:1065B600021B7222EDA2E7D2E7F9EC3340F260F358
:1065C600B4FF08ED547F70E8021B7CF82481C2E01A
:1065D600C0E0F40428FAC313FCED92E7FD9000CC6A
:1065E600121F5EEEA2E7E9BA7F02C31334009400DD
:1065F600FA75F091A4E5F013F494FE8AF0A433E55D
:10660600F033248CD313FDE492E7FE7F007C3F75C4
:106616008302ECC0E0F8EDC0E0F9EEC0E0FAEFC0AE
:10662600E0FB8583F09000CC121F0685F0831219DB
:10663600ADD0E0FBD0E0FAD0E0F9D0E0F81217B325
:10664600ED6480FD30E7011CD583C7ED33CC33F80C
:0C665600D0E0A2E71328C313CC13FD22F0
:106847009000CC121F5E9000D0E0F8A3E0F9A3E01F
:10685700FAA3E0FB9000CCE0FCA3E0FDA3E0FEA3DD
:10686700E0FF1219AD125B829000CC121F5E900000
:10687700D0E030E7599000CCE0FCA3E0FDA3E0FEB8
:10688700A3E0FFECC0E0EDC0E0EEC0E0EFC0E0E465
:10689700FFFEFDFC9000CCE0F8A3E0F9A3E0FAA32B
:1068A700E0FB121A4A7BDB600250087A0F794978BD
:1068B7004080067A0F794978C0D0E0FFD0E0FED05B
:1068C700E0FDD0E0FC1217B39000CC121F5E9000E1
:0D68D700CCE0FCA3E0FDA3E0FEA3E0FF2267
:105633003A70FA83BCAAE9E43E81E0F8BF9DE9E64B
:105643003F80000039283C1ABB9969663DA335E3C6
:10565300BF255DE73FC90FDB418DDBCCC44936EE87
:1056630045C9913FC5B0F83D3F800000C317F534ED
:10567300452FFA73C60AFDDD12573C04A2E19200DE
:105683001420E0159056337404121CC9803012574D
:105693003C30E102B20020E0EBA883A9829000CC69
:1056A300121F5E898288839056477404121CC98531
:1056B30082F09000CC121F2285F0821218A4ED4CC8
:1056C3006007300004EC6480FC2212573CC0E0A861
:1056D30083A9829000CC121F5E8982888390566BC7
:1056E3007403121CC98582F09000CC121F2285F02E
:1056F300821218A49000CCE0CCF0A3E0CDF0A3E09C
:10570300CEF0A3E0CFF090565B7403121CC9D08295
:105713008582F09000CC121F2285F082E58230E072
:10572300071219ADB2008096EFCBFFEECAFEEDC9AA
:10573300FDECC8FC1219AD8085ED33EC547FCC33FE
:10574300920024605007D0E0D0E0021B727B837A82
:10575300F97922783E1218A4EDF933ECF833248159
:105763005011EFFBEEFA121B06121AC8ECB2E7FC5B
:105773001217B3ED33EC33602F2403F8C313FCED9E
:1057830092E7FDE82481E4501FECF8EDF9EEFAEF1F
:10579300FB121B06EF04C2E0FCF582121AD2ECB234
:1057A300E7FC1217B3E58203FAED33EC3360071419
:0857B30013FCED92E7FDEA2270
:105B6200BE1249253E4CCCCDBEAAAAAB3F80000056
:105B72003E7ADBB03EED63383F24BC7D3F490FDB0C
:105B8200ED33ECC2E7CC339200B4FF13ED547F60E7
:105B920003021B727FDB7E0F7DC97C3F025C77C2F2
:105BA20001C3947F401E7007EDD2E794904015EF39
:105BB200FBEEFAEDF9ECF87F007E007D807C3F126F
:105BC20019ADD201ED33EC33248430E705E4C0E0B3
:105BD200806B04FAEDD2E754F0C333DAFD54073494
:105BE200002323C0E0CCC0E0F8EDC0E0F9EEC0E055
:105BF200FAEFC0E0FBE4121AD2EC24FEFC9000D4CF
:105C0200121F5E1218A47B007A007980783F121767
:105C1200B39000D4E0B2E7CCF0A3E0CDF0A3E0CEA5
:105C2200F0A3E0CFF0D0E0FBD0E0FAD0E0F9D0E092
:105C3200F81217B39000D4121F221219AD9000D49B
:105C4200121F5E905B627403121CC99000D4121F73
:105C5200221218A4D0E0600F246EF582E4345BF5C2
:105C620083121F2E1217B330010B7BDB7A0F79C917
:105C720078BF1217B3ED33EC336006ECA20092E763
:025C8200FC2202
:105F99009000CC121F5E74FFFFFEFDFC9000CCE068
:105FA900F8A3E0F9A3E0FAA3E0FBC3121EBB603833
:105FB9007F807E967D187C4B9000CCE0F8A3E0F9B9
:105FC900A3E0FAA3E0FB121A4A6002501B7F807E0D
:105FD900967D187CCB9000CCE0F8A3E0F9A3E0FA19
:105FE900A3E0FB121A4A500F9000CCE0FCA3E0FD9D
:105FF900A3E0FEA3E0FF229000CCE0FCA3E0FDA318
:10600900E0FEA3E0FF121B069000D0121F5E900075
:10601900D0E0FCA3E0FDA3E0FEA3E0FFEC121AC868
:10602900C8ECC8C9EDC9CAEECACBEFCB9000CCE029
:10603900FCA3E0FDA3E0FEA3E0FF1217AFE4FBFA27
:10604900F9F8121A4A602640249000D0E0FCA3E037
:10605900FDA3E0FEA3E0FFEF24FFFFEE34FFFEED1A
:1060690034FFFDEC34FFFC9000D0121F5E9000D08D
:10607900E0FCA3E0FDA3E0FEA3E0FFEC121AC822B6
:101B3D00E9D2E7C933E833F892D5EDD2E7CD33ECEE
:071B4D0033FC5002B2D52267
:101B5400EC30E7100FBF000C0EBE00080DBD0004F2
:101B64000BEB6014A2D5EB13FCED92E7FD2274FF9E
:101B7400FCFDFEFF22E480F8A2D574FF13FC7D80F7
:031B8400E480EF0B
:101B8700F920E73624F950037907E4F42402FBE54A
:101B970082158270021583DBF6E024FB501BE96097
:101BA70014E4F0E582158270021583E004F0B40AAC
:0D1BB70008E4F0D9EE7401F00A22C2D52234
:101BC400ED33EC3392D5FA602AB4FF33EDC2E77BF0
:101BD400FF60067A1B79E9E4227A1B79F220D504A6
:101BE4007A1B79ED224E614E002B494E46002D4959
:101BF4004E4600E47A08F0A3DAFC7B00740722C0A6
:101C040083C082ECC0E0EDC0E0EEC0E0EFC0E0EAEB
:101C140075F010A4CAABF075F04DA42BFBE435F0BD
:101C2400FCEA2410FAEB34C5FBEC34D9FCEDC2E732
:101C3400FF75F056A4F42411C5F0F434C58FF0A454
:101C44002AE5F03BE43CF020E714121D46D0E0FF07
:101C5400D0E0FED0E0FDD0E0FC1219AD8014F40415
:101C6400121D46D0E0FFD0E0FED0E0FDD0E0FC1233
:101C740018A4D082D083E0FAEDD2E7CD33EC33243C
:101C840082FBE4C3CF33CFCE33CECD33CD33DBF3BE
:101C94007B0775F00A846004F0A31B0AE5F0F0A347
:101CA4008FF0740AA4FFACF08EF0740AA42CFEAC7E
:101CB400F050010C8DF0740AA42CFDE435F0F0A36F
:051CC400DBDE740722C5
:101CC900C0E0EFFBEEFAEDF9ECF81218A4D0E0F55C
:101CD900F0EFFBEEFAEDF9ECF8121F12A3A3A3A3A0
:101CE900E8C0E0E9C0E0EAC0E0EBC0E0C0F01218EB
:101CF900A4121F2EA3A3A3A31217B3D0F0D0E0FB05
:0D1D0900D0E0FAD0E0F9D0E0F8D5F0D42217
:101D16003F8000004120000042C80000447A0000D5
:101D2600461C400047C35000497424004B18968057
:101D36004CBEBC205A0E1BCA6753C21C749DC5AE4E
:101D4600FB60065407601C2323121D74EB54386095
:101D560009121D60121D6F1218A4ECF8EDF9EEFAC7
:101D6600EFCB22EB121D6F80F1543803241C901D1B
:101D760016FE93FC0EEE93FD0EEE930ECE93FF220F
:1067C70002217BE493A3F8E493A34003F68001F24C
:1067D70008DFF48029E493A3F85407240CC8C333D3
:1067E700C4540F4420C8834004F456800146F6DFA2
:1067F700E4800B0102040810204080906ADEE47EEA
:10680700019360BCA3FF543F30E509541FFEE49396
:10681700A360010ECF54C025E060A840B8E493A35D
:10682700FAE493A3F8E493A3C8C582C8CAC583CA88
:10683700F0A3C8C582C8CAC583CADFE9DEE780BE40
:016B1E000076
:101D8600C2D530F707B2D563F0FF05F030E70CB2E5
:101D9600D5F4048463F0FF05F080018430D502F4A5
:021DA600042215
:101DA800BB010689828A83E0225002E722BBFE0239
:091DB800E32289828A83E493226C
:101DC100BB010CE58229F582E5833AF583E02250D7
:101DD10006E92582F8E622BBFE06E92582F8E22221
:0D1DE100E58229F582E5833AF583E493223B
:101DEE00BB010689828A83F0225002F722BBFE01D4
:021DFE00F322CE
:101E0000EF8DF0A4A8F0CF8CF0A428CE8DF0A42EF6
:021E1000FE22B0
:101E1200C2D5EC30E709B2D5E4C39DFDE49CFCEEEB
:101E220030E715B2D5E4C39FFFE49EFE12200EC335
:101E3200E49DFDE49CFC800312200E30D507C3E430
:061E42009FFFE49EFE225A
:101E4800C5F0F8A3E028F0C5F0F8E5821582700225
:061E58001583E038F022C2
:101E5E00E88FF0A4CC8BF0A42CFCE98EF0A42CFC23
:101E6E008AF0EDA42CFCEA8EF0A4CDA8F08BF0A4A1
:101E7E002DCC3825F0FDE98FF0A42CCD35F0FCEB00
:101E8E008EF0A4FEA9F0EB8FF0A4CFC5F02ECD39C5
:0F1E9E00FEE43CFCEAA42DCE35F0FDE43CFC2232
:106A5800C2D5E830E70FB2D5E4C39BFBE49AFAE469
:106A680099F9E498F8EC30E717B2D5126A8E12203B
:106A78009FE4C39BFBE49AFAE499F9E498F880034D
:106A880012209F30D50DE4C39FFFE49EFEE49DFDD8
:046A9800E49CFC225C
:0E1EAD00C3E49FFFE49EFEE49DFDE49CFC2246
:101EBB00EB9FF5F0EA9E42F0E99D42F0E89C45F07D
:011ECB0022F4
:101ECC00BB010789828A83021F065005E9F80221AB
:101EDC0031BBFE05E9F802213D89828A83021F127B
:101EEC00BB010789828A83021F5E5005E9F8022133
:0A1EFC0063BBFE05E9F802216F2226
:0C1F0600E0FCA3E0FDA3E0FEA3E0FF224E
:101F1200E493FC740193FD740293FE740393FF2215
:0C1F2200E0F8A3E0F9A3E0FAA3E0FB2242
:101F2E00E493F8740193F9740293FA740393FB2209
:101F3E00BB010789828A83021F225005E9F802211C
:101F4E0049BBFE05E9F802215689828A83021F2EBB
:0C1F5E00ECF0A3EDF0A3EEF0A3EFF022F6
:101F6A00A8828583F0D083D082121F81121F81122A
:101F7A001F81121F81E473E493A3C583C5F0C5834F
:101F8A00C8C582C8F0A3C583C5F0C583C8C582C8C1
:011F9A002224
:101F9B00F8E0FBA3A3E0F925F0F0E58215827002CF
:071FAB001583E0FA38F02273
:091FB200EBF0A3EAF0A3E9F02230
:101FBB00D083D082F8E4937012740193700DA3A3B5
:101FCB0093F8740193F5828883E4737402936860C9
:061FDB00EFA3A3A380DFC9
:101FE100D083D082F8E4937012740193700DA3A38F
:101FF10093F8740193F5828883E473740293B5F0C6
:0D200100067403936860E9A3A3A3A380D82D
:106B7F00EFB40A07740D126B8A740A309811A89932
:106B8F00B8130CC2983098FDA899C298B811F63076
:076B9F0099FDC299F599224E
:10000E00C3EE6480948040028007C3E49FFFE49EA9
:02001E00FE22C0
:10200E00BC000BBE0029EF8DF084FFADF022E4CCB6
:10201E00F875F008EF2FFFEE33FEEC33FCEE9DEC7F
:10202E00984005FCEE9DFE0FD5F0E9E4CEFD22EDC5
:10203E00F8F5F0EE8420D21CFEADF075F008EF2F0F
:10204E00FFED33FD4007985006D5F0F222C398FD00
:05205E000FD5F0EA229D
:1020630075F008758200EF2FFFEE33FECD33CDCC34
:1020730033CCC58233C5829BED9AEC99E5829840B7
:102083000CF582EE9BFEED9AFDEC99FC0FD5F0D694
:10209300E4CEFBE4CDFAE4CCF9A88222B800C1B9BE
:1020A3000059BA002DEC8BF084CFCECDFCE5F0CBFC
:1020B300F97818EF2FFFEE33FEED33FDEC33FCEB35
:1020C30033FB10D703994004EB99FB0FD8E5E4F9F0
:1020D300FA227818EF2FFFEE33FEED33FDEC33FCDD
:1020E300C933C910D7059BE99A4007EC9BFCE99AD1
:1020F300F90FD8E0E4C9FAE4CCFB2275F010EF2F16
:10210300FFEE33FEED33FDCC33CCC833C810D70715
:102113009BEC9AE899400AED9BFDEC9AFCE899F850
:0E2123000FD5F0DAE4CDFBE4CCFAE4C8F922E3
:0C213100E6FC08E6FD08E6FE08E6FF22DA
:0C213D00E2FC08E2FD08E2FE08E2FF22DE
:0D214900E6FB08E6F908E6FA08E6CBF82206
:0D215600E2FB08E2F908E2FA08E2CBF82209
:0C216300ECF608EDF608EEF608EFF622A8
:0C216F00ECF208EDF208EEF208EFF222AC
:00000001FF
